:10000000A2C20000D1C20000CFC20000CDC20000D9
:10001000CBC20000C9C20000C7C20000C5C20000B8
:10002000C3C20000C1C20000BFC20000BDC20000C8
:10003000BBC20000B9C20000B7C20000B5C20000D8
:10004000B3C200000C94D62AAFC20000ADC20000BB
:100050000C94632DA9C20000A7C200000C94822951
:10006000A3C200000C94A5270C947C279DC200001D
:100070009BC2000099C2000097C2000095C2000018
:100080000C94A92A91C200008FC200008DC200000A
:100090008BC2000089C2000087C2000085C2000038
:1000A00083C2000081C200000C947C2A7DC2000043
:1000B0007BC2000079C2000077C200000C944F2A76
:1000C00073C2000071C200006FC200006DC2000068
:1000D0006BC2000069C2000067C2000065C2000078
:1000E00063C20000E002ED02F602FF020C031503FA
:1000F000B106B106B106B106B10622032F033C03D7
:10010000B106490352035B03680371037A03830357
:100110008C039503B1069E03A703B003B106B10695
:10012000B106B903C203CB03B106B106D403E103A0
:10013000B106B106B106EE03FB030804B1061504CF
:100140001E042704B106B106B10630043904420486
:10015000B1064F045C046904B106B106B106760429
:1001600083049004B1069D04AA04B704B106B10645
:10017000B106C404D104DE04B106EB04F404FD04AA
:10018000B106B106B106B106B106B106B106B106B7
:10019000B106B106B106B106B106B106B106B106A7
:1001A000B106B106B106B106B106B106B106210528
:1001B0002A053305B1063C0545054E05B106B106D5
:1001C000B106570564057105B1067E058B059805D6
:1001D000B106B106B106A505B205BF05B106CC054D
:1001E000D505DE05B106B106B106E705F005F9054E
:1001F000B106B106B106B106B106B106B106B10647
:10020000B106B106B10606050F051805B106B1061F
:10021000B106B106B106B106B106B106B106B10626
:10022000B106B106B106B106B106B106B106B10616
:10023000B106B106B106B106B106B106B106B10606
:10024000B106B106B106B106B106B106B106B106F6
:10025000B106B106B106B106B106B106B106B106E6
:10026000B106B106B106B106B106B106B106B106D6
:10027000B106B106B10602060B061806B106250640
:100280002E063B06B106B106B106480651065E06CB
:10029000B1066B0674068106B106B106B1068E067C
:1002A0009706A406710A760A7B0A850A8F0A080B4C
:1002B000990AA10AA90AB30ABD0AC70AD60AE00A1E
:1002C000080BEA0AF40AFE0AD625D925C825CC254A
:1002D000D2251026DD25E125E725EB25EF25F5259F
:1002E000F925FD251026032607260B264E414E49EB
:1002F0004E495459494E46CDCCCC3D0AD7233C17E4
:10030000B7D13877CC2B329595E6241FB14F0A0030
:100310000020410000C84200401C4620BCBE4CCA20
:100320001B0E5AAEC59D7400407A10F35A00A0729D
:100330004E18090010A5D4E80000E8764817000020
:10034000E40B54020000CA9A3B000000E1F50500EE
:100350000080969800000040420F000000A0860137
:10036000000000102700000000E803000000006407
:1003700000000000000A0000000000010000000072
:10038000002C76D888DC674F0823DFC1DFAE59E147
:10039000B1B796E5E3E453C63AE651997696E8E6B6
:1003A000C28426EB898C9B62ED407C6FFCEFBC9C89
:1003B0009F40F2BAA56FA5F490055A2AF75C936B9B
:1003C0006CF9676DC11BFCE0E40D47FEF520E6B556
:1003D00000D0ED902E0300943577050080841E0830
:1003E0000000204E0A000000C80C333333330F984E
:1003F0006E12831141EF8D2114893BE65516CFFE15
:10040000E6DB18D1844B381BF77C1D901DA4BBE4A0
:1004100024203284725E228100C9F124ECA1E53DE2
:100420002700000A0B02090C0D0E08070304010047
:1004300000000000000000000000000000000000BC
:100440000000000000000000000000000012111079
:10045000000000000000000000000000000000009C
:100460000000000000000000002100240027002AF6
:10047000002D003000330001010000040107010AD3
:100480000100002200250028002B002E003100343E
:100490000002010000050108010B010000200023FB
:1004A00000260029002C002F00320000010000036C
:1004B00001060109010505050507050808080802E8
:1004C0000202020A0A0808040404040101010101ED
:1004D0000101010303030303030303040707070CDC
:1004E0000C0C0C0C0C0C0C02020202060606060692
:1004F0000606060B0B0B0B0B0B0B0B01021020203F
:100500000808102040102040800201020108040267
:1005100001010204081020408080402010080402DD
:100520000180040201804020100804020108040236
:10053000010102040810204080010204081020403C
:1005400080009946944611241FBECFEFD1E2DEBF52
:10055000CDBF00E00CBF17E0A0E0B2E0E0E3F1EABD
:1005600000E00BBF02C007900D92A234B107D9F78B
:100570002CE0A2E4B7E001C01D92AC3EB207E1F767
:1005800012E0C2EAD2E000E006C021970109802F04
:10059000FE010E947B4FC13AD10780E00807A9F70E
:1005A0000E944E3C0C9487502BCD603E710508F0A4
:1005B000D8C3FB018827EE58FF4F8F4F0C947B4F19
:1005C00081E090E0A0E0B0E0809356079093570759
:1005D000A0935807B0935907089510925A071092A4
:1005E0005B0710925C0710925D07089510925E07FA
:1005F00010925F071092600710926107089581E0E2
:1006000090E0A0E0B0E08093620790936307A0932E
:100610006407B09365070895109266071092670704
:100620001092680710926907089583E090E0A0E0B7
:10063000B0E080936A0790936B07A0936C07B09328
:100640006D07089588E790E0A0E0B0E0809382070E
:1006500090938307A0938407B0938507089588E754
:1006600090E0A0E0B0E08093860790938707A09386
:100670008807B0938907089588E790E0A0E0B0E08C
:1006800080938A0790938B07A0938C07B0938D0774
:100690000895109292071092930710929407109267
:1006A0009507089510929607109297071092980751
:1006B00010929907089581E090E0A0E0B0E0809367
:1006C0009A0790939B07A0939C07B0939D0708956A
:1006D00010929E0710929F071092A0071092A107F8
:1006E00008951092A2071092A3071092A4071092E7
:1006F000A50708951092A6071092A7071092A807C1
:100700001092A90708951092AA071092AB071092B1
:10071000AC071092AD0708951092AE071092AF0784
:100720001092B0071092B10708951092B20710927C
:10073000B3071092B4071092B50708951092BA0744
:100740001092BB071092BC071092BD07089510923B
:10075000BE071092BF071092C0071092C1070895FC
:100760001092C2071092C3071092C4071092C507D7
:1007700008951092D2071092D3071092D4071092C6
:10078000D50708951092D6071092D7071092D80770
:100790001092D90708951092DA071092DB07109291
:1007A000DC071092DD07089581E090E0A0E0B0E062
:1007B0008093E6079093E707A093E807B093E907D3
:1007C000089581E090E0A0E0B0E08093EA07909384
:1007D000EB07A093EC07B093ED0708958CE291E04E
:1007E000A0E0B0E08093FA079093FB07A093FC078A
:1007F000B093FD0708958CE291E0A0E0B0E0809313
:10080000FE079093FF07A0930008B0930108089596
:100810008CE291E0A0E0B0E080930208909303089E
:10082000A0930408B0930508089510920A08109246
:100830000B0810920C0810920D08089510920E08E3
:1008400010920F081092100810921108089510923B
:1008500012081092130810921408109215080895A7
:100860001092220810922308109224081092250852
:1008700008951092260810922708109228081092C6
:100880002908089581E090E0A0E0B0E080932A0874
:1008900090932B08A0932C08B0932D08089585E021
:1008A00090E0A0E0B0E08093320890933308A093EA
:1008B0003408B0933508089585E090E0A0E0B0E0FA
:1008C0008093360890933708A0933808B09339087E
:1008D000089589E190E0A0E0B0E080933A08909319
:1008E0003B08A0933C08B0933D08089582E390E054
:1008F000A0E0B0E080934A0890934B08A0934C0886
:10090000B0934D08089582E390E0A0E0B0E08093BA
:100910004E0890934F08A0935008B0935108089543
:1009200082E390E0A0E0B0E08093520890935308F7
:10093000A0935408B0935508089582E390E0A0E096
:10094000B0E080935A0890935B08A0935C08B09342
:100950005D08089582E390E0A0E0B0E080935E0837
:1009600090935F08A0936008B0936108089582E3B4
:1009700090E0A0E0B0E08093620890936308A093B9
:100980006408B0936508089580E991E0A0E0B0E0C4
:100990008093720890937308A0937408B0937508BD
:1009A000089580E991E0A0E0B0E08093760890930C
:1009B0007708A0937808B0937908089580E991E0CA
:1009C000A0E0B0E080937A0890937B08A0937C0825
:1009D000B0937D08089510928208109283081092B7
:1009E000840810928508089510928608109287084E
:1009F0001092880810928908089510928A0810921F
:100A00008B0810928C0810928D08089510929A0904
:100A100010929B0910929C0910929D0908951092C2
:100A20009E0910929F091092A0091092A1090895A1
:100A30001092A2091092A3091092A4091092A5097C
:100A400008951092EA081092EB081092EC081092A8
:100A5000ED0808951092EE081092EF081092F00839
:100A60001092F10808951092F2081092F308109273
:100A7000F4081092F50808951092FA081092FB08F5
:100A80001092FC081092FD0808951092FE08109232
:100A9000FF081092000910920109089510920209AE
:100AA000109203091092040910920509089585E037
:100AB00090E0A0E0B0E08093120990931309A09316
:100AC0001409B0931509089585E090E0A0E0B0E026
:100AD0008093160990931709A0931809B0931909E8
:100AE000089585E090E0A0E0B0E080931A0990932B
:100AF0001B09A0931C09B0931D09089584EB95E18F
:100B0000A0E0B0E08093220990932309A0932409E8
:100B1000B0932509089584EB95E1A0E0B0E08093BF
:100B2000260990932709A0932809B09329090895CD
:100B300084EB95E1A0E0B0E080932A0990932B0923
:100B4000A0932C09B0932D09089585E090E0A0E0D2
:100B5000B0E080933A0990933B09A0933C09B0938D
:100B60003D09089585E090E0A0E0B0E080933E0963
:100B700090933F09A0934009B0934109089585E0FF
:100B800090E0A0E0B0E08093420990934309A093E5
:100B90004409B0934509089510924A0910924B09EF
:100BA00010924C0910924D09089510924E0910921E
:100BB0004F0910925009109251090895109252094C
:100BC00010925309109254091092550908951092E9
:100BD00062091092630910926409109265090895E0
:100BE00010926609109267091092680910926909BB
:100BF000089510926A0910926B0910926C09109274
:100C00006D09089510927A0A10927B0A10927C0A5C
:100C100010927D0A08958CE390E0A0E0B0E080930C
:100C20007E0A90937F0AA093800AB093810A089568
:100C300081E090E0A0E0B0E08093820A9093830A84
:100C4000A093840AB093850A089510928A0A10929C
:100C50008B0A10928C0A10928D0A08958CE390E012
:100C6000A0E0B0E080938E0A90938F0AA093900A40
:100C7000B093910A089581E090E0A0E0B0E0809305
:100C8000920A9093930AA093940AB093950A0895B8
:100C90001092A20A1092A30A1092A40A1092A50A16
:100CA00008958CE390E0A0E0B0E08093A60A9093D2
:100CB000A70AA093A80AB093A90A089581E090E03A
:100CC000A0E0B0E08093AA0A9093AB0AA093AC0A8C
:100CD000B093AD0A08951092B20A1092B30A10921E
:100CE000B40A1092B50A08958CE390E0A0E0B0E059
:100CF0008093B60A9093B70AA093B80AB093B90A42
:100D0000089581E090E0A0E0B0E08093BA0A90936B
:100D1000BB0AA093BC0AB093BD0A08951092CA0AF8
:100D20001092CB0A1092CC0A1092CD0A08958CE34F
:100D300090E0A0E0B0E08093CE0A9093CF0AA09319
:100D4000D00AB093D10A089581E090E0A0E0B0E02D
:100D50008093D20A9093D30AA093D40AB093D50A71
:100D60000895660F771F660F771FFB01EA5AF84F49
:100D7000108211821282138208950F931F93CF93D2
:100D8000DF938C01C0E0D0E0BE01C8010E94F132C7
:100D9000882319F0BE01C80108DC2196C13ED105A7
:100DA00099F7DF91CF911F910F9108954F925F9224
:100DB0006F927F928F929F92AF92BF92CF92DF926B
:100DC000EF92FF92CF93DF935B01EB01CC0FDD1F1E
:100DD000CE010E94024E482E512C612C712CCE0166
:100DE00001960E94024EC82ED12CE12CF12C8DE8E8
:100DF000A81AB10883E0A816B10488F5CE0144967C
:100E00000E94024E882E912CA12CB12CCE01459629
:100E10000E94024E482F50E060E070E08FEF88168D
:100E20009104A104B104A9F44F3F51056105710576
:100E300081F48FEF481651046104710481F48FEF3F
:100E4000C816D104E104F10451F46FEF7FEFCB0138
:100E50002BC040385105610571056CF0F6CF80E874
:100E6000C816D104E104F10484F740E050E0BA016F
:100E7000812C912C5401FE2CED2CDC2CCC24C40CA8
:100E8000D51CE61CF71C540199248824C80CD91CD5
:100E9000EA1CFB1C742F662755274427CB01BA0197
:100EA0006C0D7D1D8E1D9F1DDF91CF91FF90EF90EA
:100EB000DF90CF90BF90AF909F908F907F906F907A
:100EC0005F904F9008950C94D4470C94D4470C94A1
:100ED000D447CF93DF93EB0120E030E040E85FE3BD
:100EE0006A817B818C819D810E94E64C811113C0B7
:100EF0008DE994E00E94073B0E94DF16FC01E25B53
:100F0000FF4F1082118212821382E05DFE4F108A21
:100F1000118A128A138A20E030E040E85FE36E8194
:100F20007F81888599850E94E64C811113C08DEAE6
:100F300094E00E94073B0E94DF16FC01E853FF4F3C
:100F40001082118212821382EE52FF4F108A118A90
:100F5000128A138A20E030E040E85FE36A857B85EF
:100F60008C859D850E94E64C811113C08DEB94E029
:100F70000E94073B0E94DF16FC01EE5BFE4F1082D1
:100F8000118212821382EC58FF4F108A118A128A42
:100F9000138A0E948B180E94951780E090E0DF91E1
:100FA000CF9108950F93CF93DF938091860B81119A
:100FB00076C081E08093860B0E94DF16EC0106B1BB
:100FC00026B140910001609100010295017026FB5D
:100FD000222720F941706695617082589E4F0E94C9
:100FE000863506B126B140B160B1017022FB2227DF
:100FF00020F943FB442740F966956170CE0186567F
:101000009E4F0E94863502B322B340B160B1017099
:1010100022FB222720F9441F4427441F65FB662733
:1010200060F9CE018A549E4F0E948635FE01E15937
:10103000FF4F8081882361F0709780819181A28128
:10104000B3810196A11DB11D80839183A283B383D7
:10105000FE01E751FF4F8081882361F07097808106
:101060009181A281B3810196A11DB11D80839183DD
:10107000A283B383FE01ED59FE4F8081882369F07E
:10108000CD5ADE4F88819981AA81BB810196A11D2D
:10109000B11D88839983AA83BB831092860BDF914D
:1010A000CF910F9108958F929F92AF92BF92CF925E
:1010B000DF92EF92FF920F931F930E94DF1621E0C1
:1010C0002F931F921F921F921F92812C912CA12C63
:1010D000B12CC12CD12C760197018601B701A60154
:1010E000A4D20F900F900F900F900F9080E090E09F
:1010F0001F910F91FF90EF90DF90CF90BF90AF9036
:101100009F908F900895EF92FF920F931F93CF932C
:10111000DF9300D01F92CDB7DEB78B017B01EE0CC1
:10112000FF1C622FC70129833A834B835C830E9493
:101130000A4E29813A814B815C81992757FD9A9506
:10114000852F742F632FC70101960E940A4E0D58F8
:10115000110929813A814B815C8103301105A8F482
:10116000BA01992777FD9095892FC70144960E946F
:101170000A4E29813A814B815C81652F7727882728
:101180009927C70145960E940A4E80E090E00F9093
:101190000F900F900F90DF91CF911F910F91FF90C3
:1011A000EF900895CF92DF92EF92FF92CF93DF936B
:1011B000EB010E94F132882359F1FE01EE0FFF1F6F
:1011C000EE0FFF1FEA5AF84FC080D180E280F38013
:1011D0008DEC94E00E94073B8EE496E00E94073B72
:1011E00081ED94E00E94073BCE010E947A3B8EE4A1
:1011F00096E00E94073B83ED94E00E94073BC70105
:10120000B6010E94533B0E948B180E94951704C0A0
:1012100085ED94E00E94073B80E090E0DF91CF9164
:10122000FF90EF90DF90CF900895EF92FF920F9391
:101230001F93CF93DF938091870B9091880B892B1D
:1012400009F066C084E090E00E943F47EC0160E056
:1012500070E0ACDD16161706FCF0CE018EDD96E5CB
:10126000E92E97E0F92E00E010E0B801CE010E94CF
:10127000F132882341F0F70120813181428153818D
:10128000B801CE0140DF0F5F1F4FF4E0EF0EF11CFD
:101290000639110551F738C063E070E0CE0186DDF4
:1012A000613071058105910569F586E5E82E87E0D5
:1012B000F82E00E010E0B801CE010E94F132882340
:1012C000C1F0B801CE0172DDF701608371838283C2
:1012D00093836F3F7F4F8F4F9F4F59F4B801CE01DB
:1012E00064D9F7012081318142815381B801CE0157
:1012F0000ADF0F5F1F4FF4E0EF0EF11C013E1105F6
:10130000D1F602C0CE0139DDD093880BC093870B94
:101310008091870B9091880BDF91CF911F910F9156
:10132000FF90EF900895089508950895EF92FF9229
:101330000F931F93CF93DF93162F072F7A01411539
:10134000510559F4862F0E94DB2731E020E00197F8
:1013500009F030E0C32FD22F26C04130510509F5E6
:10136000262F663310F02AEC260F80917B00922FF7
:101370009870877F892B80937B002770206420934F
:101380007C0080917A00806480937A0080917A005A
:1013900086FDFCCFC091780080917900D0E0D82BF9
:1013A00002C0C0E0D0E082E0E816F10410F587EF5B
:1013B00094E00E94073B8EE496E00E94073B81ED9B
:1013C00094E00E94073B812F902F0E947A3B8EE48D
:1013D00096E00E94073B83ED94E00E94073BCE011C
:1013E0000E947A3B0E948B180E94951780E090E043
:1013F00002C081E090E0DF91CF911F910F91FF90AB
:10140000EF9008958BEF94E00E94073B0E948B18A9
:101410000E94D21A0E948B180E94A7170E94A7341C
:1014200040E050E068E070E081DF0E94A73440E0D7
:1014300050E069E070E07ADF0E94A73440E050E0BD
:101440006AE070E073DF0E94A73440E050E06DE096
:1014500070E06CDF80E090E008950F931F93CF93CE
:10146000DF938B01EA01AB0141505109443351052F
:1014700008F0D4C02230310508F0D0C048E3429FC4
:10148000F001439FF00D1124E60FF71FE80FF91F3D
:1014900081E08083232B11F46C2F07C061E0802F43
:1014A0000E94F728209739F460E0802F0E940328DB
:1014B00080E090E0B5C0CF3FD10509F4ADC0F801A0
:1014C000EF5DFB4FE4918E2F90E0FC013197E2310C
:1014D000F10508F09DC08827EE5AFE4F8F4F0C94FF
:1014E0007B4F84B5806884BDC7BDE2CF84B5806280
:1014F00084BDC8BDDDCF809180008068809380006E
:10150000D0938900C0938800D3CF809180008062FF
:1015100080938000D0938B00C0938A00C9CF8091C4
:101520008000886080938000D0938D00C0938C00F1
:10153000BFCF8091B00080688093B000C093B300AB
:10154000B7CF8091B00080628093B000C093B400A8
:10155000AFCF80919000806880939000D0939900E5
:10156000C0939800A5CF80919000806280939000F6
:10157000D0939B00C0939A009BCF8091900088608D
:1015800080939000D0939D00C0939C0091CF809158
:10159000A00080688093A0008091A0008F7B809342
:1015A000A000D093A900C093A80082CF8091A00092
:1015B00080628093A000D093AB00C093AA0078CF44
:1015C0008091A00088608093A000D093AD00C0936C
:1015D000AC006ECF80912001806880932001D09371
:1015E0002901C093280164CF8091200180628093FB
:1015F0002001D0932B01C0932A015ACF8091200162
:10160000886080932001D0932D01C0932C0150CF8E
:10161000C038D1050CF448CF61E047CF81E090E0BD
:10162000DF91CF911F910F9108952F923F924F928A
:101630005F926F927F928F929F92AF92BF92CF9262
:10164000DF92EF92FF920F931F93CF93DF93CDB76B
:10165000DEB7E6970FB6F894DEBF0FBECDBF1C0114
:101660002A013B010B871C872D873E872E960EADE6
:101670001FAD2E97FC01E55AFD4F6081718182817B
:1016800093810E94EC4C9B01AC01C301B2010E940A
:101690004B4D0E94424F6B8B7C8B8D8B9E8BF1014F
:1016A000E15AFD4F60817181828193810E94EC4CEF
:1016B0009B01AC016B857C858D859E850E944B4D81
:1016C0000E94424F6B8F7C8F8D8F9E8FF101ED5961
:1016D000FD4F60817181828193810E94EC4C9B015E
:1016E000AC01C701B6010E944B4D0E94424F6F8F63
:1016F00078A389A39AA30E9476296B877C878D871C
:101700009E87F101E452FE4F1182108232961182BF
:1017100010823E96A114B10461F0C501A0E0B0E0D2
:10172000408151816281738184179507A607B707AD
:1017300014F0A080B180F101E051FE4F81149104BA
:1017400061F0C401A0E0B0E0408151816281738109
:1017500084179507A607B70714F080809180F101E0
:10176000EC50FE4F0115110561F0C801A0E0B0E09A
:10177000408151816281738184179507A607B7075D
:1017800014F000811181310120E1620E711CC5014C
:10179000A0E0B0E0F10180A791A7A2A7B3A7210123
:1017A000FAE84F0E511CA12CB12CD20158968D9203
:1017B0009D92AD92BC925B974101BCEF8B1ABEEF3C
:1017C0009B0A20E030E0F401008F118F228F338FCD
:1017D0000E948B180E948B180E948B180E948B18F5
:1017E00040914A0750914B0760914C0770914D070B
:1017F0004BAB5CAB6DAB7EAB0E948B1880914E0700
:1018000090914F07A0915007B09151078F87988B07
:10181000A98BBA8B0E948B18A0905207B0905307E7
:10182000C0905407D0905507F101E959FD4F10823F
:1018300011821282138234961082118212821382D4
:101840003496108211821282138234961182108291
:1018500032961182108232961182108232964BA9F2
:101860005CA96DA97EA940835183628373833496FA
:101870008F859889A989BA8980839183A283B3834C
:101880003496A082B182C282D3822F96EFAC2F977A
:101890000B891C892D893E89C3010E941C2E882337
:1018A000F9F085E393E00E94073B8AEA94E00E9406
:1018B000073BF101EE5AFF4F608171818281938174
:1018C000E75FFD4F20813181428153810E94184E94
:1018D000CA01B9010E94533B0E948B180E949517C0
:1018E0006096EFAC60970B8D1C8D2D8D3E8D4F85D6
:1018F000588969897A89C2010E941C2E8823F9F0CF
:1019000081E393E00E94073B8AEB94E00E94073B4F
:10191000F101E453FF4F6081718182819381ED5623
:10192000FE4F20813181428153810E94184ECA01AD
:10193000B9010E94533B0E948B180E949517619633
:10194000EFAC61970F8D18A129A13AA1B601A501AD
:10195000C4010E941C2E8823F9F08DE293E00E94BE
:10196000073B8AEC94E00E94073BF101EA5BFE4FE3
:101970006081718182819381E35EFE4F208131819C
:10198000428153810E94184ECA01B9010E94533B03
:101990000E948B180E949517D10151961C92F1015B
:1019A000E557FF4F1082E658FF4F1082C1010E9499
:1019B000582CC1010E945C2CC3010E946A32C201F2
:1019C0000E946A32C4010E946A32F101ED51FE4F59
:1019D000FCA3EBA381E090E0918380837101FBE1A4
:1019E000EF1AFEEFFF0AD7018D939C9381010951F5
:1019F0001E4FF8019183808341E050E0B301C101A3
:101A00000E94E318D7014D915C91B201C1010E947F
:101A1000E318F80140815181B401C1010E94E3182B
:101A200011E0F101EE53FD4F1083C3010E94092E16
:101A3000C2010E94092EC4010E94092E64E670E0D2
:101A400080E090E00E943E29C10180529E4FDC015F
:101A50001C9311961C93A1014E515E4FFA01108305
:101A60002F96FFAD2F97F1110FC060962FAD6097A5
:101A7000211105C061963FAD6197332339F1910182
:101A800021593F4FF90110826096FFAD6097F11127
:101A900005C0910127513F4FF90110826196FFADBA
:101AA0006197F11105C091012D593E4FF901108246
:101AB0002F962FAD2F97FC01208360963FAD609746
:101AC0003C936196EFAD6197DA01EC93C3010E94FC
:101AD000C52FC2010E94C52FC4010E94C52FC3019A
:101AE0000E941B2FC2010E941B2FC4010E941B2FAA
:101AF0000E948B18DC011C968C918F87A12CB12C35
:101B0000F101E052FE4FFC8BEB8B91012F513E4FC8
:101B10003C8F2B8FA1014E515E4F58A34F8FC101B7
:101B20008D519E4F9CA78BA7D101AB51BE4FBEA735
:101B3000ADA73796F8ABEFA72F5631403AA729A7A4
:101B40004F535F4F5AAB49AB8B5191409EA38DA32E
:101B5000A35AB109B8A7AFA3EB89FC898081811191
:101B60000BC0AB8DBC8D8C91811106C0EF8DF8A19F
:101B70008081882309F45DC3FF85F1115AC34BA509
:101B80005CA5B301C1010E943A194DA55EA5B20141
:101B9000C1010E943A194FA558A9B401C1010E9480
:101BA0003A19C3010E94852FC2010E94852FC401EA
:101BB0000E94852FE9A5FAA58081882321F1C30120
:101BC0000E94C52FA9A9BAA98C918823C9F06101E7
:101BD000B9E6CB1ABDEFDB0A7101EEE4EE1AEDEFC8
:101BE000FE0A81010B571D4F910127583D4FA1015E
:101BF00049595D4FB10162587E4FC3010E949C2B31
:101C0000A9A5BAA51C92F101E451FF4F8081882358
:101C100031F1C2010E94C52FF101EC55FD4F8081C9
:101C20008823C9F06101B5E6CB1ABDEFDB0A71016B
:101C3000ECE4EE1AEDEFFE0A810107571D4F91010A
:101C400023583D4FA10145595D4FB10166567E4F66
:101C5000C2010E949C2BF101E451FF4F1082F1015F
:101C6000EA59FE4F8081882331F1C4010E94C52FBB
:101C7000F101EB55FD4F80818823C9F06101F1E648
:101C8000CF1AFDEFDF0A71012AE4E21A2DEFF20A02
:101C9000810103571D4F91012F573D4FA10141591C
:101CA0005D4FB1016A547E4FC4010E949C2BF1012B
:101CB000EA59FE4F1082810101591F4FD8018C91C2
:101CC000882309F43FC0F101EF56FD4F6081718117
:101CD000072E000C880B990B0E94EC4C9B01AC0169
:101CE000F101E959FD4F60817181828193810E94E8
:101CF000734F18163CF5D8011C9264E274E0810120
:101D00000E521E4FC8010E942A2760E475E0C801E8
:101D10000E942A276CE973E0C8010E942A272F96A7
:101D2000BFAD2F97BB2309F473C3F101E258FE4FF7
:101D3000108A118A128A138AE053F14010821182AC
:101D400012821382810107511F4FF801808188237D
:101D500009F43FC0E655FE4F60817181072E000CEB
:101D6000880B990B0E94EC4C9B01AC01F101E559E9
:101D7000FD4F60817181828193810E94734F18169B
:101D800044F5F801108264E274E081010E521E4FA6
:101D9000C8010E942A2768E675E0C8010E942A2728
:101DA0006CE973E0C8010E942A276096FFAD609736
:101DB000FF2309F431C3F101E656FE4F108A118A60
:101DC000128A138AADA1BEA11D921D921D921C9272
:101DD000139781010D591E4FF8018081882309F462
:101DE0003FC0EE5CFE4F60817181072E000C880BB6
:101DF000990B0E94EC4C9B01AC01F101E159FD4FA4
:101E000060817181828193810E94734F181644F51D
:101E1000D8011C9264E274E081010E521E4FC80189
:101E20000E942A2760E975E0C8010E942A276CE910
:101E300073E0C8010E942A276196BFAD6197BB235A
:101E400009F4EEC2F101EA54FE4F108A118A128A97
:101E5000138AAFA1B8A51D921D921D921C921397D3
:101E600060E0C3010E94942E882369F0F101E25BD7
:101E7000FF4F1082118212821382E05DFE4F108AA2
:101E8000118A128A138A60E0C2010E94942E88236C
:101E900069F0EDA1FEA11082118212821382F1017C
:101EA000E656FE4F108A118A128A138A60E0C40136
:101EB0000E94942E882371F0AFA1B8A51D921D92A7
:101EC0001D921C921397F101EA54FE4F108A118A59
:101ED000128A138AF101E159FF4F8081EB89FC8955
:101EE0008083F101E751FF4F8081AB8DBC8D8C93D6
:101EF000E658FF4F8081EF8DF8A18083F101E25B0E
:101F0000FF4F20813181428153812F833887498758
:101F10005A87ADA1BEA14D915D916D917C91EFA1CC
:101F2000F8A5C080D180E280F3804BAB5CAB6DAB99
:101F30007EAB0E948B188F819885A985BA85809386
:101F40004A0790934B07A0934C07B0934D070E940C
:101F50008B184BA95CA96DA97EA940934E0750939D
:101F60004F0760935007709351070E948B18C092DF
:101F70005207D0925307E0925407F0925507C101DF
:101F80000E94582CAB89BC898C91882309F44AC0E3
:101F90000E9476292B853C854D855E8562177307E7
:101FA0008407950760F40E9476292B853C854D8532
:101FB0005E856217730784079507A0F51EC00E940F
:101FC00076296B017C012B853C854D855E85C21A87
:101FD000D30AE40AF50AF101E15BFD4F208131816A
:101FE00042815381A8EEB3E00E94344E6C157D050A
:101FF0008E059F0508F418C2D6CF0E9476296B0182
:102000007C01F101E15BFD4F2081318142815381EF
:10201000A8EEB3E00E94344E6C157D058E059F0539
:1020200008F402C2AB8DBC8D8C91882309F44AC0A0
:102030000E9476292B853C854D855E856217730746
:102040008407950760F40E9476292B853C854D8591
:102050005E856217730784079507A0F51EC00E946E
:1020600076296B017C012B853C854D855E85C21AE6
:10207000D30AE40AF50AF101ED5AFD4F20813181BE
:1020800042815381A8EEB3E00E94344E6C157D0569
:102090008E059F0508F4DEC1D6CF0E9476296B011C
:1020A0007C01F101ED5AFD4F208131814281538144
:1020B000A8EEB3E00E94344E6C157D058E059F0599
:1020C00008F4C8C1AF8DB8A18C91882309F44AC027
:1020D0000E9476292B853C854D855E8562177307A6
:1020E0008407950760F40E9476292B853C854D85F1
:1020F0005E856217730784079507A0F51EC00E94CE
:1021000076296B017C012B853C854D855E85C21A45
:10211000D30AE40AF50AF101E95AFD4F2081318121
:1021200042815381A8EEB3E00E94344E6C157D05C8
:102130008E059F0508F4A4C1D6CF0E9476296B01B5
:102140007C01F101E95AFD4F2081318142815381A7
:10215000A8EEB3E00E94344E6C157D058E059F05F8
:1021600008F48EC188EA9BE00E94E624181619063E
:1021700074F588EA9BE00E94C4248F7D8534910524
:1021800031F562E075E0C1018E529E4F0E942A2710
:1021900082E693E00E94073BBED7C7D6F101E15922
:1021A000FF4F1082E658FF4F1082E658FF4F108213
:1021B000AB89BC891C92EB8DFC8D1082AF8DB8A1D0
:1021C0001C92B1E0BF87AA24A394B12C03C0A11430
:1021D000B10481F067E175E0C1018E529E4F0E940B
:1021E0002A27EB89FC891082AB8DBC8D1C92EF8D68
:1021F000F8A11082C1010E94BD3AF101E252FE4FE6
:10220000808191810196918380838D3291400CF47D
:10221000A3CCD101AA52BE4F8D919C911197892BCD
:1022200009F09ACC14968D919C91892B09F43EC1AA
:1022300093CC81010A521E4FD8018D919C91892B1C
:1022400021F0C1010E94BD3AF7CF87E295E00E94DC
:10225000073B2F96BFAD2F97BB23E9F0A114B10424
:10226000D1F4EF85E1113AC08DE193E00E94073B84
:1022700052D75BD66096FFAD6097FF2351F189E19D
:1022800093E00E94073B47D750D661962FAD6197E8
:10229000211118C023C060963FAD6097332339F0F9
:1022A000A114B10421F44F85411118C0E8CF619603
:1022B0005FAD6197552391F0A114B10479F48F8536
:1022C00081110CC085E193E00E94073B24D72DD6F5
:1022D00005C06196EFAD6197E111F4CF85E090E024
:1022E000ABA1BCA18D939C9391012B513E4F3C8798
:1022F0002B87D9018D939C93810109511E4FF801C1
:102300009183808345E050E0B301C1015CD7AB8588
:10231000BC854D915C91B201C10155D7F801408156
:102320005181B401C1014FD7C1010E94602CF1015C
:10233000E25BFF4F4081518162817381E658FF4F1C
:1023400080819181A281B3818F8B988FA98FBA8F61
:10235000E658FF4FC080D180E280F3804BAB5CAB8E
:102360006DAB7EABD8D64BA95CA96DA97EA9409375
:102370004A0750934B0760934C0770934D07CBD699
:102380002F89388D498D5A8D20934E0730934F07F2
:102390004093500750935107BED6C0925207D09237
:1023A0005307E0925407F0925507C1010E94582C40
:1023B000C1010E945C2CAFD60BD6C10193D7ABA153
:1023C000BCA11D921C92EB85FC8511821082D80164
:1023D0001D921C9240E050E0B301C101F4D6EB85A0
:1023E000FC8540815181B201C101EDD6D8014D91EA
:1023F0005C91B401C101E7D6C1010E94602CBF8588
:10240000BB2309F44DC187D621E0FC01248748C1D4
:10241000AA24A394B12C96CCAA24A394B12CD9CCF1
:10242000AA24A394B12C1CCD69E273E081010E5261
:102430001E4FC8010E942A276CE973E0C8010E9460
:102440002A2768EB75E0C8010E942A2722E0A22E05
:10245000B12CE8CD65E273E081010E521E4FC80138
:102460000E942A276CE973E0C8010E942A276DECBC
:1024700075E0C8010E942A2792E0A92EB12C22CE35
:1024800061E273E081010E521E4FC8010E942A27AB
:102490006CE973E0C8010E942A2762EE75E0C8016A
:1024A0000E942A2782E0A82EB12C5CCE11821082D5
:1024B000F101E452FE4F80819181009749F46EE56D
:1024C00073E081010E521E4FC8010E942A27C5C029
:1024D000019709F0D1C01FD68C01FC018081918148
:1024E000A281B381181619061A061B0644F081E072
:1024F00090E0A0E0B0E080839183A283B383F801F1
:1025000084819581A681B781181619061A061B06C3
:1025100044F081E090E0A0E0B0E084839583A6835E
:10252000B783F80180859185A285B38518161906B1
:102530001A061B0644F081E090E0A0E0B0E080873E
:102540009187A287B3876EE973E0CE0101960E945E
:10255000682763E275E0CE0101960E942A276AEAA5
:1025600074E0CE0101960E942A2760914A0770917B
:102570004B0780914C0790914D070E94EC4C6B01EA
:102580007C01D8016D917D918D919C910E94EC4CC4
:102590009B01AC01C701B6010E94DA4EAB01BC0140
:1025A000CE0101960E94FA266AEB74E0CE010196F4
:1025B0000E942A2760914E0770914F078091500723
:1025C000909151070E94EC4C6B017C01F8016481F1
:1025D0007581868197810E94EC4C9B01AC01C701FB
:1025E000B6010E94DA4EAB01BC01CE0101960E94F9
:1025F000FA266AEC74E0CE0101960E942A276091C7
:1026000052077091530780915407909155070E948B
:10261000EC4C6B017C01D80118966D917D918D91E8
:102620009C911B970E94EC4C9B01AC01C701B60129
:102630000E94DA4EAB01BC01CE0101960E94FA263F
:10264000BE016F5F7F4F81010E521E4FC8010E9475
:10265000382789819A810E94D4475DD5BC01CE017B
:1026600001961DD4BE016F5F7F4FC8010E943827BD
:1026700089819A810E94D447F101E452FE4F808102
:1026800091810196823091051CF49183808302C070
:1026900011821082F101E652FE4F118210825CCA53
:1026A00085E395E00E94073BC5010E947A3B8CE9D7
:1026B00093E00E94073B2FD5B0924507A0924407B4
:1026C000C501E6960FB6F894DEBF0FBECDBFDF9111
:1026D000CF911F910F91FF90EF90DF90CF90BF901F
:1026E000AF909F908F907F906F905F904F903F90B2
:1026F0002F900895662319F08DEA93E002C086EAD0
:1027000093E00C94073B0C94D4470C94D447AF92BD
:10271000BF92CF92DF92EF92FF920F931F93CF93CE
:10272000DF93EC0186E390E09E8B8D8B87E390E056
:10273000988F8F8B86E290E09A8F898F8AE190E064
:102740009C8F8B8F8CE190E09E8F8D8F88E190E045
:1027500098A38F8F83E090E09AA389A382E090E012
:102760009CA38BA3FE01E657FF4F8CE390E096837A
:1027700085838DE390E09087878388E390E092875C
:1027800081871486138616861586108A17868EE032
:1027900090E0928B818B8FE090E0948B838BE65856
:1027A000FF4F8EE290E09683858380E390E09087F0
:1027B00087838EE390E0928781871486138616863E
:1027C0001586108A178682E190E0928B818B83E1D7
:1027D00090E0948B838BE152FF4F118210823296EE
:1027E00011821082329611821082CE010E94291D20
:1027F000CE0154D76E0182E8C81A8EEFD80AAA24F7
:10280000A394B12CF601B38EA28E7E01F6E6EF1AE8
:10281000FEEFFF0A84E090E0F701938F828F8E0134
:102820000A541E4F88E090E0F801938F828F80E178
:1028300090E0F6019183808381E190E09583848329
:102840008FE190E09383828381E290E09783868397
:10285000C6010E944F35F601828580878385818776
:1028600087E190E0F7019183808389E190E095838F
:10287000848383E290E09383828385E290E0978370
:102880008683C7010E944F35F70182858087838543
:1028900081878BE190E0F801918380838DE190E066
:1028A0009583848387E290E09383828389E290E03A
:1028B00097838683C8010E944F35F80182858087FF
:1028C00083858187EE5FFE4F808191813C972081D7
:1028D0003181369740815181F601578B468B358B7C
:1028E000248B019729F48FEF9FEF918F808F03C086
:1028F000F601B18EA08EFE01E654FD4F80819181DC
:102900003C9720813181369740815181F701578B67
:10291000468B358B248B019719F48FEF9FEF03C003
:1029200081E090E0F701918F808FFE01E454FD4F2C
:10293000808191813C9720813181C655DD4F48814E
:102940005981F801578B468B358B248B019719F4ED
:102950008FEF9FEF03C081E090E0F801918F808FAF
:10296000DF91CF911F910F91FF90EF90DF90CF906B
:10297000BF90AF9008952F923F924F925F926F92C7
:102980007F928F929F92AF92BF92CF92DF92EF92FF
:10299000FF920F931F93CF93DF93CDB7DEB7CA5744
:1029A000D1090FB6F894DEBF0FBECDBF8C01FC017C
:1029B000108211821282138214821582168217826B
:1029C000108611861286138614861586168617863B
:1029D0002C01F0E14F0E511CC2010E948C326801A3
:1029E0008AE8C80ED11CC6010E948C327801ECEF37
:1029F000EE1AEEEFFE0AC7010E948C323801F2E8AF
:102A00006F1AFEEF7F0AC3010E94D535480186E6A2
:102A1000881A8EEF980AC4010E94D5355801EAE45D
:102A2000AE1AEEEFBE0AC5010E94D5356EE973E01D
:102A3000C8018E529E4F0E946827F801E852FE4F4F
:102A40001182108232961182108232961182108287
:102A5000329611821082329610823196108231960F
:102A60001082319611821082329611821082329633
:102A70001182108232961082319610823196108225
:102A80003196108211821282138234961082118242
:102A9000128213823496108211821282138234962B
:102AA0001082118212821382349610821182128255
:102AB000138234961082118212821382349610820D
:102AC0001182128213823496108211821282138232
:102AD00034961082118212821382349610821182EF
:102AE00012821382349610821182128213823496DB
:102AF0001082118212821382349610821182128205
:102B000013823496108211821282138234961082BC
:102B1000118212821382349610823196108231967D
:102B200010823196108211821282138234961082A2
:102B300011821282138234961082118212821382C1
:102B4000349610823196108231961082319610821E
:102B50003196108231961082319610823196108211
:102B60003196108231961082319610823196108201
:102B700031961082319610823196108231961082F1
:102B800031961082319610823196108231961082E1
:102B900031961082319610823196108231961082D1
:102BA0003196108211821282138234961082118221
:102BB0001282138234961082118212821382D801FB
:102BC000A55ABD4F8CE0E9E3F3E001900D928A95A0
:102BD000E1F7F801E959FD4F108211821282138248
:102BE00034961082118212821382349610821182DE
:102BF00012821382349611821082329611821082D0
:102C000032961182108232961082118212821382C1
:102C100034961082118212821382349610821182AD
:102C20001282138234961082118212821382349699
:102C300010821182128213823496108211821282C3
:102C4000138234961182108232961182108232964B
:102C5000118210823296108211821282138234966F
:102C60001082118212821382349610821182128293
:102C700013823496108231961082319610823196EA
:102C80001182108232961182108232961182108245
:102C900032961182108232961182108232961182FF
:102CA00010823296118210823296118210823296F0
:102CB0001182108232961182108232961182108215
:102CC00032961182108232961182108232961182CF
:102CD00010821801FEE32F1AFDEF3F0AF101108266
:102CE000CE0101960E948C328AE7FE013196D20114
:102CF00001900D928A95E1F7CE0101960E948C32E7
:102D00008AE7FE013196D60101900D928A95E1F78E
:102D1000CE0101960E948C328AE7FE013196D701DE
:102D200001900D928A95E1F788E5F801808B89E59D
:102D3000F60180838AE5F7018083CE0101960E9427
:102D4000D5358CE1FE013196D30101900D928A9523
:102D5000E1F7CE0101960E94D5358CE1FE01319656
:102D6000D40101900D928A95E1F7CE0101960E945F
:102D7000D5358CE1FE013196D50101900D928A95F1
:102D8000E1F7C801C4DCF1011082C658DF4F0FB66D
:102D9000F894DEBF0FBECDBFDF91CF911F910F9191
:102DA000FF90EF90DF90CF90BF90AF909F908F906B
:102DB0007F906F905F904F903F902F900895CF93AA
:102DC000DF938091930B9091940B892B51F483ECBA
:102DD00092E00E943F47EC01CEDDD093940BC0936C
:102DE000930B8091930B9091940BDF91CF91089569
:102DF0004F925F926F927F928F929F92AF92BF920B
:102E0000CF92DF92EF92FF920F931F93CF93DF93B6
:102E100000D01F92CDB7DEB7FB01168907898288E3
:102E20009388A684B784C284D384E484F5844680DE
:102E300057806084718442815381648175814983A4
:102E40005A836B837C83BBDF1F921F921F920F9369
:102E50001F939301820149815A816B817C810E9479
:102E6000150B0F900F900F900F900F9080E090E057
:102E70000F900F900F900F90DF91CF911F910F91B6
:102E8000FF90EF90DF90CF90BF90AF909F908F908A
:102E90007F906F905F904F90089508950895EF92FE
:102EA000FF920F931F93CF93DF93CDB7DEB72E978B
:102EB0000FB6F894DEBF0FBECDBF8C016EE973E094
:102EC0000E94682767EF75E0C8010E942A27609179
:102ED00046077091470780914807909149072AE07B
:102EE000AE014F5F5F4F7A010E94A348F701019046
:102EF0000020E9F73197AF014E195F09B701C8010A
:102F00000E94CD266CE973E0C8010E942A27C801FF
:102F10002E960FB6F894DEBF0FBECDBFDF91CF91D6
:102F20001F910F91FF90EF90089587EF95E00E9419
:102F3000073B609146077091470780914807909141
:102F400049070E94533B8CE993E00C94073B0F9395
:102F50001F93CF93DF93EC018AEF95E00E94073B2C
:102F60008EEF95E00E94073B0DE81BE0F8016081C1
:102F7000CE01C0DB82E096E00E94073BF801618150
:102F8000CE01B8DB86E096E00E94073BF801628143
:102F9000CE01B0DB8AE096E00E94073BF801638136
:102FA000CE01A8DB8EE096E00E94073BF801648129
:102FB000CE01A0DB82E196E00E94073BF80165812B
:102FC000CE0198DBCE01DF91CF911F910F91ADCF54
:102FD000CF92DF92EF92FF92CF93DF93EC01888143
:102FE0009981AA81BB81181619061A061B0644F09E
:102FF00081E090E0A0E0B0E088839983AA83BB835E
:103000008C819D81AE81BF81181619061A061B0698
:1030100044F081E090E0A0E0B0E08C839D83AE833B
:10302000BF8388859985AA85BB85181619061A0657
:103030001B0644F081E090E0A0E0B0E0888799872B
:10304000AA87BB8783E295E00E94073B8AEA94E067
:103050000E94073B60914A0770914B0780914C0793
:1030600090914D070E94EC4C6B017C016881798145
:103070008A819B810E94EC4C9B01AC01C701B60187
:103080000E94DA4E42E00E947F3B8AEB94E00E946D
:10309000073B60914E0770914F07809150079091C8
:1030A00051070E94EC4C6B017C016C817D818E810B
:1030B0009F810E94EC4C9B01AC01C701B6010E94AC
:1030C000DA4E42E00E947F3B8AEC94E00E94073B8C
:1030D0006091520770915307809154079091550762
:1030E0000E94EC4C6B017C01688579858A859B8503
:1030F0000E94EC4C9B01AC01C701B6010E94DA4E64
:1031000042E00E947F3BCE01DF91CF91FF90EF9094
:10311000DF90CF900ACF80918B0B90918C0B892BF5
:1031200091F58DE090E00E943F47FC0114861092DB
:103130004A0710924B0710924C0710924D071092BD
:103140004E0710924F07109250071092510710929D
:10315000520710925307109254071092550710927D
:103160008A0B1092890B1092460710924707109213
:103170004807109249071092450710924407909310
:103180008C0B80938B0B80918B0B90918C0B089503
:103190000F931F93CF93DF938B01EA0181E593E0B7
:1031A0000E94073B8EE496E00E94073BF801808175
:1031B0000E94483BCE010E947A3BADDFDF91CF9168
:1031C0001F910F91B2CECF92DF92EF92FF920F93A9
:1031D0001F93CF93DF93CDB7DEB728970FB6F89440
:1031E000DEBF0FBECDBF8B016A018E529E4F7C01A8
:1031F0006DE473E00E942A276EE476E0C7010E9426
:103200002A27F801808189831A8241E050E08E01EB
:103210000F5F1F4FB801C7010E94CD264AE0B801D9
:10322000C6010E949948F80101900020E9F7319702
:10323000AF01401B510BB801C7010E94CD266BDFC7
:10324000BC01C8012CDEB801C7010E943827898162
:103250009A810E94D44728960FB6F894DEBF0FBE1D
:10326000CDBFDF91CF911F910F91FF90EF90DF9035
:10327000CF900895FC01DB01AD59BF4F8C9188239D
:1032800019F022E030E002C020E030E0DB01AB5971
:10329000BF4F8C91882311F023E030E0DB01AC5963
:1032A000BF4F8C91882311F024E030E0DB01AA5954
:1032B000BF4F8C91882311F026E030E0DA018D9128
:1032C0009C918217930721F091E0121613060CF0DF
:1032D00090E0DA012D933C93992319F0A901CF01D5
:1032E00072CF08958F929F92AF92BF92CF92DF924A
:1032F000EF92FF920F931F93CF93DF93EC0189E43A
:1033000093E00E94073B8AEA94E00E94073B6E012B
:1033100082E8C81A8EEFD80AC6010E94B5350E940D
:10332000EC4C4B015C01FE01E55AFD4F608171815F
:10333000828193810E94EC4C9B01AC01C501B401D8
:103340000E94DA4E42E00E947F3B8AEB94E00E94AA
:10335000073B7E01E6E6EE1AEEEFFE0AC7010E9489
:10336000B5350E94EC4C4B015C01FE01E15AFD4F6A
:1033700060817181828193810E94EC4C9B01AC0140
:10338000C501B4010E94DA4E42E00E947F3B8AEC04
:1033900094E00E94073B8E010A541E4FC8010E9410
:1033A000B5350E94EC4C4B015C01CD59DD4F688175
:1033B00079818A819B810E94EC4C9B01AC01C50103
:1033C000B4010E94DA4E42E00E947F3BA4DEADDDF4
:1033D00085E493E00E94073B8AEA94E00E94073B61
:1033E000F601A08DB18D20893189428953890E94CF
:1033F0003E4E0E94533B8AEB94E00E94073BF7014C
:10340000A08DB18D20893189428953890E943E4E19
:103410000E94533B8AEC94E00E94073BF801A08D88
:10342000B18D20893189428953890E943E4E0E9484
:10343000533B71DEDF91CF911F910F91FF90EF9081
:10344000DF90CF90BF90AF909F908F906ECD4F92B6
:103450005F926F927F928F929F92AF92BF92CF9224
:10346000DF92EF92FF920F931F93CF93DF9300D0E1
:103470001F92CDB7DEB70E941509409032085090D8
:10348000330860903408709035080E9415098090C8
:10349000360890903708A0903808B09039083BDE85
:1034A000C0904A07D0904B07E0904C07F0904D0732
:1034B00032DEC701B6010E94EC4C6B017C01C301F6
:1034C000B2010E94EC4C9B01AC01C701B6010E9405
:1034D000DA4E2B013C0160914E0770914F078091AD
:1034E0005007909151070E94EC4C6B017C01C50183
:1034F000B4010E94EC4C9B01AC01C701B6010E94D3
:10350000DA4EAB01BC0149835A836B837C8357DC61
:103510001F921F921F921F921F92812C912CA12CFF
:10352000B12CC12CD12C760149815A816B817C81CF
:103530008A019B01B301A2010E94150B40DC1F927E
:103540001F921F921F921F9297018601B301A20141
:103550000E94150B34DC1F921F921F921F921F9224
:1035600097018601B701A6010E94150B0FB6F894CA
:10357000DEBF0FBECDBF80E090E00F900F900F90A8
:103580000F90DF91CF911F910F91FF90EF90DF90FF
:10359000CF90BF90AF909F908F907F906F905F90F3
:1035A0004F900895CF93DF9383E00E94DB27EC01D7
:1035B000B2DD91E0CD2B09F490E090938D0B82E089
:1035C0000E94DB27EC01A7DD91E0CD2B09F490E010
:1035D00090938E0B8EE00E94DB27EC019CDD91E046
:1035E000CD2B09F490E090938F0B8FE00E94DB27A6
:1035F000EC0191DD91E0CD2B09F490E09093900BDC
:1036000082E10E94DB27EC0186DD91E0CD2B09F4FD
:1036100090E09093910B83E10E94DB27EC017BDD2E
:1036200091E0CD2B09F490E09093920BDF91CF9134
:103630000895CF93DF93EC012AEC30E04BEC50E09F
:1036400069EC70E00E944D2B2EEC30E04FEC50E026
:103650006DEC70E0CE010C960E944D2B24ED30E015
:1036600045ED50E063ED70E0CE0148960E944D2B91
:1036700028ED30E049ED50E067ED70E0CE01849632
:103680000E944D2B2EED30E04FED50E06DED70E0DF
:10369000CE01C096DF91CF910C944D2B2F923F928B
:1036A0004F925F926F927F928F929F92AF92BF9252
:1036B000CF92DF92EF92FF920F931F93CF93DF93FE
:1036C000EC010E941509FE01EF56FD4F8091120991
:1036D00090911309918380830E941509FE01ED5694
:1036E000FD4F8091160990911709918380830E9464
:1036F0001509FE01EB56FD4F80911A0990911B09A7
:10370000918380830E9415098E0109561D4F609197
:103710003A0970913B0980913C0990913D090E94C2
:10372000EC4CF80160837183828393830E941509B6
:103730001E01F5E62F1AFDEF3F0A60913E097091D8
:103740003F0980914009909141090E94EC4CF101A0
:1037500060837183828393830E94150920E030E0A7
:1037600048EC52E4F80160817181828193810E946A
:10377000DA4E2B013C0120E030E048EC52E4F1014C
:1037800060817181828193810E94DA4E4B015C01DC
:1037900060914209709143098091440990914509D3
:1037A0000E94EC4C20E030E048EC52E40E94DA4EFB
:1037B0006B017C012AE037ED43E25CE3C301B20117
:1037C0000E94734F18168CF420E030E046EC52E46F
:1037D000C301B2010E94E64C87FD0FC0412C512C61
:1037E00046EC642E42E4742E08C05AE0452E57ED94
:1037F000552E53E2652E5CE3752EF801408251820E
:10380000628273822AE037ED43E25CE3C501B401D2
:103810000E94734F18168CF420E030E046EC52E41E
:10382000C501B4010E94E64C87FD0FC0812C912C8C
:1038300026ECA22E22E4B22E08C03AE0832E37ED09
:10384000932E33E2A32E3CE3B32EF10180829182CA
:10385000A282B3822AE037ED43E25CE3C701B601FE
:103860000E94734F18168CF420E030E046EC52E4CE
:10387000C701B6010E94E64C87FD0FC0C12CD12CB8
:1038800086ECE82E82E4F82E08C09AE0C92E97ED67
:10389000D92E93E2E92E9CE3F92EFE01E156FD4F6D
:1038A000C082D182E282F3820E9415098091FA08D7
:1038B0009091FB08FE01EA55FD4F918380830E94A1
:1038C00015098091FE089091FF08FE01E855FD4F13
:1038D000918380830E9415098091020990910309C8
:1038E000FE01E655FD4F918380830E94150980916A
:1038F000220990912309FE01E455FD4F91838083B5
:103900000E9415098091260990912709FE01E25530
:10391000FD4F918380830E94150980912A0990911F
:103920002B09FE01E055FD4F918380830E9415090C
:1039300080914A0990914B09FE01EE54FD4F91830D
:1039400080830E94150980914E0990914F09FE01D4
:10395000EC54FD4F918380830E9415098091520998
:1039600090915309FE01EA54FD4F918380830E9498
:1039700015098091620990916309FE01E854FD4F99
:10398000918380830E94150980916609909167094F
:10399000FE01E654FD4F918380830E9415098091BA
:1039A0006A0990916B09FE01E454FD4F9183808375
:1039B0000E9415098091EA089091EB08A091EC080B
:1039C000B091ED08FE01ED55FD4F0197A105B10540
:1039D00019F481E0808301C010820E941509809152
:1039E000EE089091EF08A091F008B091F108FE0167
:1039F000EC55FD4F0197A105B10519F481E08083D5
:103A000001C010820E9415098091F2089091F3087C
:103A1000A091F408B091F508CB55DD4F0197A105B1
:103A2000B10519F481E0888301C01882DF91CF913C
:103A30001F910F91FF90EF90DF90CF90BF90AF90CC
:103A40009F908F907F906F905F904F903F902F90BE
:103A500008952F923F924F925F926F927F928F9232
:103A60009F92AF92BF92CF92DF92EF92FF920F930D
:103A70001F93CF93DF93CDB7DEB760970FB6F8945F
:103A8000DEBF0FBECDBF988B8F870E941509EF85D3
:103A9000F889E751FE4F81E04091220850912308B8
:103AA0006091240870912508452B462B472B09F47B
:103AB00080E080830E941509EF85F889E651FE4F6A
:103AC00081E0409126085091270860912808709164
:103AD0002908452B462B472B09F480E080830E9460
:103AE0001509EF85F889E551FE4F81E040912A08DC
:103AF00050912B0860912C0870912D08452B462B76
:103B0000472B09F480E080830E9415098091720898
:103B100090917308A0917408B0917508EF85F889A9
:103B2000E451FE4F80839183A283B3830E941509E1
:103B30008091760890917708A0917808B0917908E3
:103B4000EF85F889E051FE4F80839183A283B38390
:103B50000E94150980917A0890917B08A0917C08B9
:103B6000B0917D08EF85F889EC50FE4F80839183FA
:103B7000A283B3830E94150980914A0890914B0853
:103B8000A0914C08B0914D08EF85F889EC5FFD4F8E
:103B900080839183A283B3830E94150980914E088C
:103BA00090914F08A0915008B0915108EF85F88985
:103BB000E85FFD4F80839183A283B3830E94150940
:103BC0008091520890915308A0915408B0915508E3
:103BD000EF85F889E45FFD4F80839183A283B383EF
:103BE0000E94150980915A0890915B08A0915C0889
:103BF000B0915D08EF85F889E05FFD4F8083918388
:103C0000A283B3830E94150980915E0890915F089A
:103C1000A0916008B0916108EF85F889EC5EFD4FD6
:103C200080839183A283B3830E94150980916208E7
:103C300090916308A0916408B0916508EF85F889B8
:103C4000E85EFD4F80839183A283B3830E941509B0
:103C50008091FA079091FB07A091FC07B091FD07B6
:103C6000EF85F889E45EFD4F80839183A283B3835F
:103C70000E9415098091FE079091FF07A09100080E
:103C8000B0910108EF85F889E05EFD4F8083918354
:103C9000A283B3830E9415098091020890910308C2
:103CA000A0910408B0910508EF85F889EC5DFD4FFF
:103CB00080839183A283B3830E941509EF85F889DD
:103CC000E85DFD4F81E02091D2073091D30721308C
:103CD000310509F080E080830E941509EF85F8899D
:103CE000E75DFD4F81E02091D6073091D707213065
:103CF000310509F080E080830E941509EF85F8897D
:103D0000E65DFD4F81E02091DA073091DB0721303D
:103D1000310509F080E080830E941509EF85F8895C
:103D2000EA5BFD4F81E04091AA075091AB0760919B
:103D3000AC077091AD07452B462B472B09F480E06B
:103D400080830E941509EF85F889E95BFD4F81E0CA
:103D50004091AE075091AF076091B0077091B107E5
:103D6000452B462B472B09F480E080830E941509E0
:103D7000EF85F889E85BFD4F81E04091B2075091F3
:103D8000B3076091B4077091B507452B462B472BBD
:103D900009F480E080830E941509EF85F889E75BCC
:103DA000FD4F81E040918208509183086091840822
:103DB00070918508452B462B472B09F480E08083C2
:103DC0000E941509EF85F889E65BFD4F81E040917F
:103DD0008608509187086091880870918908452B62
:103DE000462B472B09F480E080830E941509EF855C
:103DF000F889E55BFD4F81E040918A0850918B087E
:103E000060918C0870918D08452B462B472B09F447
:103E100080E080830E941509EF85F889E45BFD4FFF
:103E200081E02091BA073091BB072130310509F0BC
:103E300080E080830E941509EF85F889E35BFD4FE0
:103E400081E02091BE073091BF072130310509F094
:103E500080E080830E941509EF85F889E25BFD4FC1
:103E600081E02091C2073091C3072130310509F06C
:103E700080E080830E9415098091820790918307DA
:103E8000A0918407B0918507EF85F889E15BFD4F2C
:103E900080839183A283B3830E9415098091860752
:103EA00090918707A0918807B0918907EF85F889DD
:103EB000ED5AFD4F80839183A283B3830E9415093D
:103EC00080918A0790918B07A0918C07B0918D0704
:103ED000EF85F889E95AFD4F80839183A283B383EC
:103EE0000E941509EF85F889E65CFD4F81E040915D
:103EF0009207509193076091940770919507452B15
:103F0000462B472B09F480E080830E941509EF853A
:103F1000F889E55CFD4F81E0409196075091970745
:103F20006091980770919907452B462B472B09F410
:103F300080E080830E941509EF85F889E45CFD4FDD
:103F400081E040919A0750919B0760919C07709186
:103F50009D07452B462B472B09F480E080830E9468
:103F6000150980918A0990918B09A0918C09B091D3
:103F70008D09EF85F889E55DFD4F80839183A283EC
:103F8000B3830E94150980918E0990918F09A091A9
:103F90009009B0919109EF85F889E15DFD4F80832B
:103FA0009183A283B3830E94150980919209909115
:103FB0009309A0919409B0919509EF85F889ED5C7A
:103FC000FD4F80839183A283B3830E941509EF85FF
:103FD000F889E35CFD4F81E02091EA073091EB071F
:103FE0002130310509F080E08083EF85F889E25CBB
:103FF000FD4F1082EF85F889E15CFD4F10820E9431
:104000001509EF85F889E05CFD4F81E02091E60716
:104010003091E7072130310509F080E08083EF859A
:10402000F889EF5BFD4F1082EF85F889EE5BFD4F5D
:1040300010820E941509EF85F889ED5BFD4F81E044
:1040400020910A0830910B082130310509F080E0F9
:1040500080830E941509EF85F889EC5BFD4F81E0B4
:1040600020910E0830910F082130310509F080E0D1
:1040700080830E941509EF85F889EB5BFD4F81E095
:1040800020911208309113082130310509F080E0A9
:1040900080830E941509EF85F889E95CFD4F81E076
:1040A00020919A0930919B092130310509F080E077
:1040B00080830E941509EF85F889E85CFD4F81E057
:1040C00020919E0930919F092130310509F080E04F
:1040D00080830E941509EF85F889E75CFD4F81E038
:1040E0002091A2093091A3092130310509F080E027
:1040F00080830E9415090F851889055A1D4F8091EC
:10410000320890913308A0913408B0913508F80135
:1041100080839183A283B3830E941509EF84F8887A
:10412000F1EAEF1AFDEFFF0A809136089091370807
:10413000A0913808B0913908F70180839183A28358
:10414000B3830E94150980913A0890913B08A09191
:104150003C08B0913D082F8538892D593D4FF90114
:1041600080839183A283B383F8014081518162816E
:104170007381141615061606170644F041E050E048
:1041800060E070E04083518362837383F701408174
:10419000518162817381141615061606170644F0C4
:1041A00041E050E060E070E04083518362837383BC
:1041B000181619061A061B064CF081E090E0A0E0E4
:1041C000B0E0F90180839183A283B383D9018D90FC
:1041D0009D90AD90BC90F701C080D180E280F380CB
:1041E000D8014D905D906D907C900E948B18FC01E1
:1041F0004082518262827382C482D582E682F782D3
:1042000080869186A286B386EF85F889E95CFD4FAA
:10421000B081B983EF85F889E55DFD4F808191819B
:10422000A281B3814F8558894D5B5D4FFA01F081C2
:10423000FB834F855889445B5D4FFA01F081FA8317
:104240004F855889435C5D4FFA01F081FF834F85AC
:104250005889405C5D4FFA01F081F8874F85588995
:10426000475B5D4FFA01F081F9874F8558894A5BBA
:104270005D4FFA01F081FA87EF85F889E85DFD4F1F
:104280002080EF85F889E751FE4F3080EF85F8896F
:10429000E15BFD4F4081518162817381EF85F88937
:1042A000E45EFD4F0081118122813381EF85F88921
:1042B000E05FFD4FC080D180E280F380EF85F88918
:1042C000EC5FFD4F80809180A280B380EF85F889FC
:1042D000E451FE4F4080518062807380EF85F88901
:1042E00040A651A662A673A684A695A6A6A6B7A6C2
:1042F000C0AAD1AAE2AAF3AA04AB15AB26AB37AB8E
:1043000040AF51AF62AF73AF34AE25AE2A8525A35F
:10431000398536A34A8147A340E450E060E070E06D
:10432000E05CFF4F40835183628373832885EF8570
:10433000F88926AF3F8137AFAF014C5B5F4F2B81D0
:10434000FA012083EF85F889EB5BFF4F808391832F
:10435000A283B383EF85F889E75BFF4F3981308310
:10436000AF85B88955968D919C9156978633910566
:1043700089F483EA9CE2FD01E658FF4F9183808334
:1043800032961182108281EA9CE236969183808374
:10439000329630C08C33910589F48BE99CE2EF852D
:1043A000F889E658FF4F91838083EF85F889E458B8
:1043B000FF4F1182108289E99CE212C08E97E1F4CE
:1043C00083E99CE2EF85F889E658FF4F918380836B
:1043D000EF85F889E458FF4F118210828DE89CE246
:1043E000EF85F889EE57FF4F91838083EF85F88939
:1043F000EC57FF4F11821082EF85F889838D948DE1
:104400004A97D1F48FE99CE2E258FF4F9183808371
:10441000EF85F889E058FF4F118210828DE99CE208
:10442000EF85F889EA57FF4F91838083EF85F889FC
:10443000E857FF4F11821082EF85F889E85CFD4F45
:1044400020812983EF85F889E15DFD4F408051800F
:1044500062807380EF85F889EC5BFD4F30813B8390
:10446000EF85F889E35BFD4F9081EF85F889E25C89
:10447000FD4F40814F83EF85F889EF5BFD4F508101
:104480005887EF85F889E65BFD4F8081EF85F889D5
:10449000E95BFD4FA081AA87EF85F889E75DFD4FB5
:1044A0002080EF85F889E651FE4F3080EF85F8894E
:1044B000ED5AFD4F20813181428153812B873C870A
:1044C0004D875E87EF85F889E05EFD4F4081518121
:1044D00062817381EF85F889EC5EFD4FC080D180E9
:1044E000E280F380EF85F889E85FFD4F808091805E
:1044F000A280B380EF85F889E657FF4F2F85388972
:1045000020513E4FD9010D911D912D913C91008F6D
:10451000118F228F338F848E958EA68EB78EC0A278
:10452000D1A2E2A2F3A244A355A366A377A32B854D
:104530003C854D855E8520A731A742A753A734A6A9
:1045400025A63A85358B868B978B80E490E0A0E09A
:10455000B0E080AB91ABA2ABB3AB488546A75F811F
:1045600057A78B8184AB45AA56AA67AA70AE9981DA
:1045700091AF858196818633910589F483EA9CE227
:10458000AF85B889AC50BF4F8D939C93AF85B889E8
:10459000AA50BF4F1D921C9281EA9CE226C08C3328
:1045A000910589F48BE99CE2AF85B889AC50BF4F87
:1045B0008D939C93AF85B889AA50BF4F1D921C92D2
:1045C00089E99CE212C08E97E1F483E99CE2AF8511
:1045D000B889AC50BF4F8D939C93AF85B889AA50D2
:1045E000BF4F1D921C928DE89CE2AF85B889A45004
:1045F000BF4F8D939C93AF85B889A250BF4F1D923A
:104600001C92838594854A97D9F48FE99CE2EF85C3
:10461000F889E850FF4F91838083EF85F889E65051
:10462000FF4F118210828DE99CE2EF85F889F395A6
:1046300091838083EF85F889EE5FFE4F11821082AF
:10464000EF85F889E75CFD4FA081A9832F85388924
:104650002D5C3D4FD9018D919D910D90BC91A02D68
:104660008B839C83AD83BE83EF85F889EB5BFD4F25
:10467000B081BA83EF85F889E25BFD4F20812F83FB
:10468000EF85F889E15CFD4F30813887EF85F88947
:10469000EE5BFD4F40814987EF85F889E55BFD4F73
:1046A0002080EF85F889E85BFD4F3080EF85F88941
:1046B000E65DFD4F3081EF85F889E551FE4F2081A1
:1046C000EF85F889E95AFD4F80819181A281B381FC
:1046D000EF85F889EC5DFD4F4081518162817381E6
:1046E000EF85F889E85EFD4FC080D180E280F380DD
:1046F000EF85F889E45FFD4F80809180A280B380D0
:104700000F8518890C5F1E4FEF85F889EC50FE4F1E
:104710004080518062807380F801408E518E628E9D
:10472000738E848E958EA68EB78EC0A2D1A2E2A281
:10473000F3A244A355A366A377A380A791A7A2A73A
:10474000B3A724A735A7358A268A2F81278B80E433
:1047500090E0A0E0B0E080AB91ABA2ABB3AB298519
:1047600026A7388537A74A8144AB8B819C81AD81D0
:10477000BE8185AB96ABA7ABB0AF298121AF858158
:1047800096818633910589F483EA9CE2EF85F88966
:10479000E259FE4F91838083EF85F889E059FE4FFF
:1047A0001182108281EA9CE226C08C33910589F443
:1047B0008BE99CE2EF85F889E259FE4F9183808373
:1047C000EF85F889E059FE4F1182108289E99CE259
:1047D00012C08E97E1F483E99CE2EF85F889E259F3
:1047E000FE4F91838083EF85F889E059FE4F118257
:1047F00010828DE89CE2EF85F889EA58FE4F91839C
:104800008083EF85F889E858FE4F11821082D80125
:104810001B968D919C911C974A97E1F48FE99CE23D
:10482000EF85F889EE58FE4F91838083EF85F889F4
:10483000EC58FE4F118210828DE99CE2EF85F889D9
:10484000E658FE4F91838083EF85F889E458FE4F48
:1048500011821082EF85F889E65CFD4F20818F85FB
:1048600098894096222319F00E94092E02C00E94C6
:10487000F72DEF85F889E55CFD4F20818F859889BC
:1048800086579F4F222319F00E94092E02C00E94D2
:10489000F72DEF85F889E45CFD4F80818823D9F0FE
:1048A000C80160960FB6F894DEBF0FBECDBFDF9192
:1048B000CF911F910F91FF90EF90DF90CF90BF901D
:1048C000AF909F908F907F906F905F904F903F90B0
:1048D0002F900C94092EC80160960FB6F894DEBF95
:1048E0000FBECDBFDF91CF911F910F91FF90EF9041
:1048F000DF90CF90BF90AF909F908F907F906F9000
:104900005F904F903F902F900C94F72DCF92DF92B5
:10491000EF92FF920F931F93CF93DF936C017A0175
:104920008B01C0E0D0E0CE15DF0589F0D8016D9194
:104930008D01D601ED91FC910190F081E02DC60131
:104940001995892B11F47E0102C02196ECCFC70185
:10495000DF91CF911F910F91FF90EF90DF90CF905B
:104960000895089580E090E00895FC01538D448DF2
:10497000252F30E0842F90E0821B930B541710F00A
:10498000CF96089501970895FC01918D828D981717
:1049900061F0828DDF01A80FB11D5D968C91928D23
:1049A0009F5F9F73928F90E008958FEF9FEF089520
:1049B000FC01918D828D981731F0828DE80FF11DE9
:1049C000858D90E008958FEF9FEF0895FC01918D04
:1049D000228D892F90E0805C9F4F821B91098F73FD
:1049E0009927089588EA9BE0F1DF21E0892B09F4FB
:1049F00020E0822F0895FC01848DDF01A80FB11DF6
:104A0000A35ABF4F2C91848D90E001968F73992704
:104A1000848FA689B7892C93A089B1898C918064F1
:104A20008C93938D848D981306C00288F389E02DB2
:104A300080818F7D80830895EF92FF920F931F9363
:104A4000CF93DF93EC0181E0888F9B8D8C8D981341
:104A500005C0E889F989808185FD23C0F62E0B8D7C
:104A600010E00F5F1F4F0F731127E02E8C8DE8129F
:104A70000BC00FB607FCFACFE889F989808185FF62
:104A8000F5CFCE01B8DFF2CF8B8DFE01E80FF11D1F
:104A9000E35AFF4FF0820B8FEA89FB8980818062A5
:104AA00007C0EE89FF896083E889F9898081806485
:104AB000808381E090E0DF91CF911F910F91FF9073
:104AC000EF900895CF93DF93EC01888D8823C1F098
:104AD000EA89FB89808185FD05C0A889B9898C9107
:104AE00086FD0EC00FB607FCF5CF808185FFF2CFA3
:104AF000A889B9898C9185FFEDCFCE017CDFE8CF05
:104B0000DF91CF91089580E090E0892B19F06ADF62
:104B1000811125C080E090E0892B41F080E090E099
:104B2000892B21F00E94000081111CC080E090E0E0
:104B3000892B41F080E090E0892B21F00E94000059
:104B4000811113C080E090E0892BA1F080E090E01B
:104B5000892B81F00E94000081110AC008950E94F3
:104B60000000D8CF0E940000E1CF0E940000EACFF1
:104B70000C940000089590E0FC013197E231F105BA
:104B800008F04EC08827EC59FE4F8F4F0C947B4F96
:104B9000809180008F7703C0809180008F7D80930B
:104BA0008000089580918000877FF9CF84B58F774A
:104BB00002C084B58F7D84BD08958091B0008F7749
:104BC00003C08091B0008F7D8093B00008958091E4
:104BD00090008F7707C0809190008F7D03C08091F7
:104BE0009000877F8093900008958091A0008F7738
:104BF00007C08091A0008F7D03C08091A000877FB7
:104C00008093A0000895809120018F7707C0809144
:104C100020018F7D03C080912001877F8093200138
:104C200008953FB7F89480919E0B90919F0BA091AF
:104C3000A00BB091A10B26B5A89B05C02F3F19F082
:104C40000196A11DB11D3FBFBA2FA92F982F88270C
:104C5000820F911DA11DB11DBC01CD0142E0660F67
:104C6000771F881F991F4A95D1F708950E946A50AF
:104C70000C94D4470C94D4470F931F93CF93DF9396
:104C8000EC0188819981009729F02A813B812617C0
:104C9000370788F48B016F5F7F4F0E94834F009727
:104CA00061F0998388831B830A832C813D81232BA8
:104CB00011F4FC01108281E001C080E0DF91CF910E
:104CC0001F910F9108958F929F92AF92BF92CF92B2
:104CD000DF92EF92FF920F931F930E94DF1662E024
:104CE00070E00E94F535892BD1F40E94DF1621E097
:104CF0002F931F921F921F921F92812C912CA12CF7
:104D0000B12CC12CD12C760197018601B701A601E7
:104D10000E94150B0F900F900F900F900F9080E056
:104D200090E01F910F91FF90EF90DF90CF90BF9098
:104D3000AF909F908F9008958F929F92AF92BF9265
:104D4000CF92DF92EF92FF920F931F930E94DF1694
:104D50001F9221E02F931F921F921F92812C912C62
:104D6000A12CB12CC12CD12C760197018601B70161
:104D7000A6010E94150B0F900F900F900F900F90AF
:104D800080E090E01F910F91FF90EF90DF90CF9027
:104D9000BF90AF909F908F900895EF92FF920F93E6
:104DA0001F93CF93DF93FC01248135816115710539
:104DB00011F480E018C041155105A1F07B01EC0110
:104DC0008A01020F131FB80157DF882391F328814E
:104DD00039818C819D81B701820F931F0E94805081
:104DE0001D830C8381E0DF91CF911F910F91FF9084
:104DF000EF900895EF92FF920F931F93CF93DF935D
:104E0000CDB7DEB764970FB6F894DEBF0FBECDBF47
:104E10007C01CB01BA018E010F5F1F4F22E044E0FD
:104E20000E942047BC01FC0101900020E9F7319766
:104E3000AF01481B590BC701B0DF64960FB6F89459
:104E4000DEBF0FBECDBFDF91CF911F910F91FF90BD
:104E5000EF9008956115710549F0FB010190002064
:104E6000E9F73197AF01461B570B97CF80E00895C4
:104E7000FB0144815581608171818FCFEF92FF9258
:104E80000F931F93CF93DF93EC017B018A01BA014B
:104E9000F3DE2881398181110DC02115310519F00A
:104EA000C9010E94D447198218821D821C821B826C
:104EB0001A8206C01D830C83B701C9010E9480506D
:104EC000CE01DF91CF911F910F91FF90EF90089548
:104ED000FC011182108213821282158214826115E4
:104EE000710549F0FB0101900020E9F73197AF010E
:104EF000461B570BC3CF08951F920F920FB60F9208
:104F000011240BB60F922F933F934F935F936F93A0
:104F10007F938F939F93AF93BF93EF93FF9388EA11
:104F20009BE069DDFF91EF91BF91AF919F918F91D0
:104F30007F916F915F914F913F912F910F900BBE99
:104F40000F900FBE0F901F9018951F920F920FB6E3
:104F50000F9211240BB60F922F938F939F93EF9381
:104F6000FF93E091B80BF091B90B8081E091BE0BFB
:104F7000F091BF0B82FD12C090818091C10B8F5FB9
:104F80008F732091C20B821751F0E091C10BF0E0BA
:104F9000E855F44F958F8093C10B01C08081FF913C
:104FA000EF919F918F912F910F900BBE0F900FBE9D
:104FB0000F901F901895CF93DF93282F30E0F901C1
:104FC000EF5DFB4F8491F901E550FB4FD491F9015E
:104FD000EB54FB4FC491CC2389F08111CCDDEC2F35
:104FE000F0E0EE0FFF1FE556FB4FA591B491EC9159
:104FF000ED2381E090E021F480E002C080E090E0C9
:10500000DF91CF9108951F93CF93DF93282F30E046
:10501000F901EF5DFB4F8491F901E550FB4FD4910D
:10502000F901EB54FB4FC491CC23C1F0162F811131
:10503000A2DDEC2FF0E0EE0FFF1FEF57FB4FA59125
:10504000B4918FB7F894111105C09C91ED2FE095A4
:10505000E92302C0EC91ED2BEC938FBFDF91CF9150
:105060001F910895CF92DF92EF92FF920F931F93BB
:10507000CF93DF936C018B017A01EC01CB56D44FB7
:10508000888187FF04C0FB011182108224C08CE05C
:105090008C9D90018D9D300D11248881A901480FB0
:1050A000511D87FD5A958091DD0C90E048175907F6
:1050B00094F48881A901480F511D87FD5A95CA01B2
:1050C000FA01EE0FFF1F8E0F9F1FFC01E35BF34FF2
:1050D000808186FD19C088818F5F88838CE08C9DDC
:1050E00090018D9D300D11248881A901480F511D1B
:1050F00087FD5A958091DD0C90E048175907B4F46C
:1051000088818C303CF112C08881280F311D87FDC9
:105110003A95F901EE0FFF1F2E0F3F1FF901E35BD8
:10512000F34F808160E08F736EDFD5CFF80180810F
:105130009181049680349C4918F480E49CE904C071
:10514000F801808191810496F701918380838FEF2C
:10515000888344C0F801408151818881B901680F7A
:10516000711D87FD7A95CB01FB01EE0FFF1F8E0F9E
:105170009F1FFC01E35BF34F81819281840F951F98
:10518000F701918380838881A901480F511D87FD14
:105190005A95CA01FA01EE0FFF1F8E0F9F1FFC01E7
:1051A000E35BF34F808186FF19C08881280F311D92
:1051B00087FD3A95F901EE0FFF1F2E0F3F1FF901F2
:1051C000E35BF34F808161E08F73DF91CF911F919B
:1051D0000F91FF90EF90DF90CF9015CFDF91CF919F
:1051E0001F910F91FF90EF90DF90CF900895CF9394
:1051F000DF9390E0FC01E550FB4F2491FC01EB5460
:10520000FB4F8491882361F190E0880F991FFC0186
:10521000E959FB4FC591D491FC01EF57FB4FA59184
:10522000B491611109C09FB7F894888120958223B9
:105230008883EC912E230BC0623061F49FB7F89401
:105240003881822F809583238883EC912E2B2C9399
:105250009FBF06C08FB7F894E8812E2B28838FBF9D
:10526000DF91CF9108958230910538F0880F991F12
:10527000880F991F05970197F1F708958F929F92D4
:10528000AF92BF92CF92DF92EF92FF926B017C01BF
:10529000C8DC4B015C01C114D104E104F104E9F064
:1052A000C0DCDC01CB0188199909AA09BB09883E39
:1052B0009340A105B10578F321E0C21AD108E108B5
:1052C000F10888EE880E83E0981EA11CB11CC11461
:1052D000D104E104F10421F7DECFFF90EF90DF90DD
:1052E000CF90BF90AF909F908F9008952FB7F89474
:1052F00060919A0B70919B0B80919C0B90919D0BF0
:105300002FBF08951F920F920FB60F9211242F9363
:105310003F938F939F93AF93BF9380919A0B9091FC
:105320009B0BA0919C0BB0919D0B3091990B23E0AE
:10533000230F2D3720F40196A11DB11D05C026E8CD
:10534000230F0296A11DB11D2093990B80939A0BF8
:1053500090939B0BA0939C0BB0939D0B80919E0B05
:1053600090919F0BA091A00BB091A10B0196A11D54
:10537000B11D80939E0B90939F0BA093A00BB093B5
:10538000A10BBF91AF919F918F913F912F910F9062
:105390000FBE0F901F901895CF92DF92EF92FF9261
:1053A000CF93DF93EC01603282E078070CF03DC0D0
:1053B00077FD06C0653B71052CF064EB70E002C020
:1053C00060E070E0898128E830E06901C81AD108FE
:1053D00087FDD394CC0CDD1CCC0CDD1C0D2C000CFB
:1053E000EE08FF088A8128E532E0281B310987FD95
:1053F0003395220F331F220F331FC901330FAA0B1E
:10540000BB0B9C01AD012C193D094E095F09DB0165
:105410000E943E4E24EB30E040E050E00E94184EE7
:10542000C20ED31EE41EF51EB6018881803380F5BE
:10543000998148E850E0491B510997FD5395440F65
:10544000551F440F551F6417750784F09A8128E58E
:1054500032E0291B310997FD3395220F331F220FAC
:10546000331FAB01261737070CF4A901425051092D
:10547000440F551F2FB7F89490E0FC01EE0FFF1F6B
:105480008E0F9F1FFC01E35BF34F528341832FBFBD
:10549000DF91CF91FF90EF90DF90CF9008951F9212
:1054A0000F920FB60F9211240BB60F922F933F93CA
:1054B0004F935F936F937F938F939F93AF93BF931C
:1054C000EF93FF9348E251E064E271E080E090E006
:1054D000C9DDFF91EF91BF91AF919F918F917F9126
:1054E0006F915F914F913F912F910F900BBE0F9055
:1054F0000FBE0F901F9018951F920F920FB60F922C
:1055000011240BB60F922F933F934F935F936F939A
:105510007F938F939F93AF93BF93EF93FF9348EA4B
:1055200050E064EA70E083E090E09CDDFF91EF9151
:10553000BF91AF919F918F917F916F915F914F91AB
:105540003F912F910F900BBE0F900FBE0F901F90A9
:1055500018951F920F920FB60F9211240BB60F924F
:105560002F933F934F935F936F937F938F939F936B
:10557000AF93BF93EF93FF9348E950E064E970E085
:1055800082E090E06FDDFF91EF91BF91AF919F912D
:105590008F917F916F915F914F913F912F910F90DC
:1055A0000BBE0F900FBE0F901F9018951F920F9279
:1055B0000FB60F9211240BB60F922F933F934F9378
:1055C0005F936F937F938F939F93AF93BF93EF936B
:1055D000FF9348E850E064E870E081E090E042DD4D
:1055E000FF91EF91BF91AF919F918F917F916F91BB
:1055F0005F914F913F912F910F900BBE0F900FBE77
:105600000F901F90189508950F931F93CF93DF93DA
:10561000FC012081318121153105D1F1EC01822F6E
:10562000CADC21E0892B09F420E02B876A85261744
:1056300029F01E821F82188619860BC08E819F81D9
:10564000A885B9850196A11DB11D8E839F83A8876A
:10565000B9870E811F81288539858A819B81AC811C
:10566000BD81081719072A073B0794F081E06827D6
:105670008881C9DC0990D881C02D0E94A73440E000
:1056800050E0BE01DF91CF911F910F910C949609CC
:10569000DF91CF911F910F910895CF92DF92EF92FA
:1056A000FF920F931F93CF93DF937C016B018A01CD
:1056B000E9010E941509F601EE0FFF1FEE0FFF1F13
:1056C000EA5AF84F80819181F701918380830E948B
:1056D0001509000F111F000F111FF801EA5AF84FAA
:1056E00081E04081518162817381413051056105C2
:1056F000710509F080E0F70182870E941509CC0F3F
:10570000DD1FCC0FDD1FCA5AD84F88819981AA812D
:10571000BB81F70182839383A483B58316821782AA
:1057200010861186DF91CF911F910F91FF90EF901E
:10573000DF90CF90089508952F923F924F925F92FD
:105740006F927F928F929F92AF92BF92CF92DF9291
:10575000EF92FF920F931F93CF93DF9300D000D06F
:10576000CDB7DEB79E838D834B015A013A832983DF
:105770001801FC82EB82FA014080518062807380C4
:1057800020E030E0A901C301B2010E94734F181656
:1057900074F4F6012081318142815381C301B20149
:1057A0000E94754EF5016083718382839383ED813E
:1057B000FE81E05AFF4F8081F401008D118DC08879
:1057C000D188E288F388F101408051806280738043
:1057D000D801A7019601882341F00E943E4E64152E
:1057E00075058605970544F023C00E943E4E461677
:1057F000570668067906E4F4F5014080518062801E
:10580000738020E030E04AEF56E4C301B2010E9409
:10581000E64C87FF0DC020E030E040E85FE3C301C5
:10582000B2010E94764EF501608371838283938377
:10583000D801A70196010E943E4EF1016083718359
:10584000828393830D811E81025C1F4FF80180814A
:105850009181A281B381E981FA8180839183A283BE
:10586000B383EB81FC8180819181892B41F0C4015C
:105870000E94B535F80160837183828393832696F5
:105880000FB6F894DEBF0FBECDBFDF91CF911F9151
:105890000F91FF90EF90DF90CF90BF90AF909F90CF
:1058A0008F907F906F905F904F903F902F900895D2
:1058B0000E948B180C94D21A0E948B180C94A71774
:1058C000CF93DF93EC01FC01EE53FD4F1082E858BB
:1058D000F1098081811103C0CE01409688D1FE017B
:1058E000E55CFD4F8081811104C0CE0186579F4F3A
:1058F0007ED1FE01E45CFD4F8081811104C0CE01A8
:105900008C5F9E4F74D164E670E080E090E0DF91A0
:10591000CF91B4CC8FEF9FEF0895EBE0F1E0808161
:10592000877F80830895EBE0F1E080818860808349
:1059300008958E9808958E9A089514980895149A4B
:10594000089588980895889A08950C94D4470C94E3
:10595000D4470C94D4470C94D4470C94D4470F9359
:105960001F93CF93DF93FB01C2A1D3A1068D178DA7
:105970008091A20B9091A30B892B41F481E090E0E0
:105980000E943F479093A30B8093A20B0430110514
:1059900039F00530110541F4BE0181EE9CE003C0F1
:1059A000BE018EED9CE0F8DC80E090E0DF91CF91CD
:1059B0001F910F9108958F929F92AF92BF92CF92B5
:1059C000DF92EF92FF920F931F930E94DF161F92B8
:1059D0001F9221E02F931F921F92812C912CA12CBA
:1059E000B12CC12CD12C760197018601B701A601FB
:1059F0000E94150B0F900F900F900F900F9080E06A
:105A000090E01F910F91FF90EF90DF90CF90BF90AB
:105A1000AF909F908F9008950E948B180E94E81776
:105A200080E090E0089560E0FC018385ECCA60E0CE
:105A3000FC018581E8CA61E0FC018385E4CA61E07C
:105A4000FC018581E0CACF93DF93FB01C68DD78D22
:105A50000E941509BE010E94D20880E090E0DF910B
:105A6000CF910895CF93DF938091A40B9091A50BD4
:105A7000892BF1F48CE390E00E943F47EC01FC019C
:105A8000CC96118210823C96E817F907D1F719825B
:105A900018821D861C86198E188E1DA21CA219AA9A
:105AA00018AACE010E94191BD093A50BC093A40B7A
:105AB0008091A40B9091A50BDF91CF91089508954B
:105AC0000895089508951F920F920FB60F92112412
:105AD0000BB60F922F933F934F935F936F937F93E8
:105AE0008F939F93AF93BF93EF93FF93E091420700
:105AF000F09143071995FF91EF91BF91AF919F915D
:105B00008F917F916F915F914F913F912F910F9066
:105B10000BBE0F900FBE0F901F901895CF93DF9381
:105B2000EC01FC01E759FF4F1082379781E0808339
:105B300060E08D8168DA8F859889892B29F060E093
:105B40008B85DF91CF915FCADF91CF910895CF937D
:105B5000DF93EC018B892FDA2E8930E082179307CF
:105B600011F48F8901C080E0DF91CF910895CF9328
:105B7000DF93EC0189891FDA2E8930E082179307C1
:105B800011F48F8901C080E0DF91CF910895CF9308
:105B9000DF93EC018DA5882311F061E001C060E086
:105BA0008F8131DA8EA5882329F08FA5882311F003
:105BB00061E001C060E08D85DF91CF9124CACF9371
:105BC000DF93EC018DA5882311F060E001C061E056
:105BD0008F8119DA8EA5882329F08FA5882311F0EB
:105BE00060E001C061E08D85DF91CF910CCACF9359
:105BF000DF93EC0161E0898506DA8EA5882319F030
:105C000061E08F8500DAC959DF4F1882DF91CF91AB
:105C10000895CF93DF93EC0160E08985F4D98EA5D8
:105C2000882319F060E08F85EED9C959DF4F81E0F4
:105C30008883DF91CF910895CF92DF92EF92FF9208
:105C40000F931F93CF93DF93FC0142AF53AF64AF29
:105C500075AFDC01DE964D935D936D937C93139746
:105C600014960D931D932D933C931397EC01CA5BEF
:105C7000DF4FE88284A9882389F084A5811109C0B7
:105C800037FF0CC01D921D921D921C92139781E04C
:105C900006C01016110612061306A4F380E045A9EB
:105CA00056A967A970AD14161506160617063CF519
:105CB00091AD992321F10D911D912D913C91139757
:105CC0006801790137FF07C0CC24DD247601C01AB2
:105CD000D10AE20AF30A4C155D056E057F057CF4D6
:105CE00037FF07C070956095509541955F4F6F4F96
:105CF0007F4F4D935D936D937C93139781E0DF010C
:105D0000A15BBF4F1D921D921D921C921397E15AE9
:105D1000FF4F91E09083DF91CF911F910F91FF9002
:105D2000EF90DF90CF9008950F931F93CF93DF9361
:105D30008C01D62FFC018589811109C0C80117DFAC
:105D4000C82FC80104DFD11108C08C2F06C0C801BC
:105D5000FEDEC82FC8010BDFF6CFDF91CF911F9178
:105D60000F910895CF93DF93EC01FC01E759FF4FAA
:105D700081E0808339978081B297882341F08081C8
:105D80009181A281B3810196A11DB11D07C08081BF
:105D90009181A281B3810197A109B1098083918387
:105DA000A283B383FE01E459FF4F20813181DE01DC
:105DB000A659BF4FC9019595879520FD03C0ED9168
:105DC000FC910DC0FE01E80FF91F0190F081E02D5C
:105DD0002D913C91E20FF31F0190F081E02D8C0F8B
:105DE0009D1F19958F859889892B11F1FE01E05926
:105DF000FF4F20813181DE01A259BF4FC901959526
:105E0000879520FD03C0ED91FC910DC0FE01E80FC8
:105E1000F91F0190F081E02D2D913C91E20FF31FCD
:105E20000190F081E02D8C0F9D1FDF91CF9119948F
:105E3000DF91CF9108958F929F92AF92BF92CF92B0
:105E4000DF92EF92FF920F931F93CF93DF93EC01BA
:105E5000FC01E15BFF4F60817181828193810E942F
:105E6000EA4C6B017C0168A979A98AA99BA90E94C7
:105E7000EC4C9B01AC0160E074E284E799E40E9481
:105E8000DA4E4B015C01FE01E55AFF4F60817181E2
:105E9000828193810E94EA4C9B01AC01C501B4014F
:105EA0000E94DA4E4B015C018E010D5A1F4F20E01B
:105EB00030E040E05FE30E944B4D9B01AC01C70125
:105EC000B6010E94764E0E94474FF80160837183AD
:105ED00082839383C95ADF4FA5019401C701B6019C
:105EE0000E94764E0E94474F688379838A839B8302
:105EF000DF91CF911F910F91FF90EF90DF90CF90A6
:105F0000BF90AF909F908F9008950F931F93CF9362
:105F1000DF93FC01E759FF4F20812223B9F07A97E4
:105F200000811181228133813896408151816281C3
:105F30007381041715072607370710F1EC01EEDD12
:105F4000CE01DF91CF911F910F9175CFFC01E15AE6
:105F5000FF4F20812223A1F07097008111812281BF
:105F60003381349640815181628173810417150712
:105F70002607370728F0DF91CF911F910F91F2CEBE
:105F8000DF91CF911F910F9108952F923F924F92E1
:105F90005F926F927F928F929F92AF92BF92CF92B9
:105FA000DF92EF92FF920F931F93CF93DF93CDB7C2
:105FB000DEB762970FB6F894DEBF0FBECDBF8C017F
:105FC0007C0126E4E20EF11CD7018C919801205A45
:105FD0003F4FF801EF59FF4F6F01A801425C5F4F3F
:105FE0004A0114971D01882341F0F80184A5D901C5
:105FF0008C9381E0F60180832FC0DA014D915D9191
:106000006D917C91F10180819181A281B381BB244A
:10601000B394481759076A077B070CF0B12CF901B4
:10602000B08277FF07C070956095509541955F4F9E
:106030006F4F7F4FB7FF07C0B095A09590958195A2
:106040009F4FAF4FBF4F21E0481759076A077B07A3
:106050000CF420E0D6012C93F4014081518162813F
:106060007381411551056105710559F4F801848D5D
:10607000958DA68DB78DE55AFF4F80839183A283BE
:10608000B383F10180819181A281B381F80142AC97
:1060900053AC64AC75AC9801215A3F4F5901481676
:1060A00059066A067B0634F4481759076A077B07C6
:1060B0007CF00AC084159505A605B7052CF4841755
:1060C0009507A607B70724F0D7018C918823D9F04C
:1060D000F50180818823B9F0D7018C91811105C029
:1060E000F701808181110FC006C060E0C8011CDE8D
:1060F0008111F6CF17C0D6016C9181E06827C801E5
:1061000013DE882379F0D5011C9260E0C8010CDE13
:10611000882309F4C6C1F801FE961082118212820A
:106120001382BFC1D80194962D913D914D915C9100
:10613000979729833A834B835C8358962D913D91A1
:106140004D915C915B972D833E834F8358875C967E
:106150002D913D914D915C915F9729873A874B87AF
:106160005C87F10180819181A281B381F801FE9663
:10617000C080D180E280F380F80142AD53AD64ADC0
:1061800075ADED59FF4F1082319610823801F5E65A
:106190006F0E711CF301108298012A593F4FF901CB
:1061A0001082329610824C015D01841A950AA60A6B
:1061B000B70AB7FE08C0B094A09490948094811C54
:1061C000911CA11CB11C481759076A077B072CF4C6
:1061D000C41AD50AE60AF70A04C0C81AD90AEA0A94
:1061E000FB0AD501C401B595A795979587958D872D
:1061F0009E87AF87B88BD801A859BF4F1D01F7FC08
:1062000005C08C149D04AE04BF044CF4F80100A03A
:10621000F1A1E02DFA8BE98B81E0D9011BC02D851E
:106220003E854F8558892C153D054E055F0508F4C0
:1062300054C089819A81AB81BC818C159D05AE05C6
:10624000BF0564F42D813E812F5F3F4F3A8B298B30
:1062500081E0D3018C93F10180839EC0C701B60118
:106260000E94EC4C2B013C0169817A818B819C81DD
:106270000E94EC4C9B01AC01C301B2010E94DA4EBA
:106280002B013C016D817E818F81988529853A851E
:106290004B855C85621B730B840B950B0E94EC4C49
:1062A0009B01AC01C301B2010E944B4D2B013C018B
:1062B00069857A858B859C850E94EC4C9B01AC019D
:1062C000C301B2010E94764E0E94424F7A8B698BC5
:1062D00081E0F801ED59FF4F5CC0D501C40129816F
:1062E0003A814B815C81821B930BA40BB50BC816C2
:1062F000D906EA06FB065CF42D813E812E5F3F4FF6
:106300003A8B298B81E0F801EB59FF4F42C0C50160
:10631000B4016C197D098E099F090E94EC4C2B0178
:106320003C0169817A818B819C810E94EC4C9B01AC
:10633000AC01C301B2010E94DA4E2B013C016D8118
:106340007E818F81988529853A854B855C85621B86
:10635000730B840B950B0E94EC4C9B01AC01C301A9
:10636000B2010E944B4D2B013C0169857A858B85DA
:106370009C850E94EC4C9B01AC01C301B2010E94C0
:10638000764E0E94424F7A8B698B81E0F801EC597E
:10639000FF4F8083D1018C93F80184818823B1F071
:1063A0000E947629D80112964D905C901397052C87
:1063B000000C66087708DC01CB0184199509A60951
:1063C000B709893E9340A105B10568F4F801E55A83
:1063D000FF4F29893A89C901A0E0B0E08083918309
:1063E000A283B38392CE0E947629D80113967C9320
:1063F0006E93129784E294E00E94073B86E196E058
:106400000E94073B60E070E0CB010E94533B8CE1AF
:1064100096E00E94073BC701B6010E94533B82E20F
:1064200096E00E94073BC501B4010E94533B88E2FD
:1064300096E00E94073B4AE06D857E858F859889AE
:106440000E94083B8FE296E00E94073B69817A81B7
:106450008B819C810E94533B85E396E00E94073B21
:1064600069857A858B859C850E94533B8BE396E0FA
:106470000E94073B6D817E818F8198850E94533BEE
:1064800081E496E00E94073B8EE496E00E94073B81
:1064900089899A890E947A3B8CE993E00E94073BA4
:1064A00095CF62960FB6F894DEBF0FBECDBFDF91D9
:1064B000CF911F910F91FF90EF90DF90CF90BF9001
:1064C000AF909F908F907F906F905F904F903F9094
:1064D0002F9008950F931F93FC01EA5BFF4F2081DB
:1064E000211110C0389700811181228133813496A7
:1064F0004081518162817381041715072607370790
:1065000044F404C0FC0124A5222319F01F910F912B
:1065100056CB1F910F913BCBFC0113821282148248
:1065200016821582108617821286118614861386AB
:1065300016861586108A1786128A118A148A138A7B
:10654000DC01A15ABF4F1C9212AE13AE14AE15AEB1
:1065500091971D921D921D921C92139714961D9255
:106560001D921D921C92139714961C925A961C927F
:1065700011961C9212961C9211961C9211961C92C6
:1065800011961C9211961C9211961C9211961C92B7
:1065900011968FE19DE211969C938E93129611961F
:1065A0001C921E9212968BE19DE211969C938E9303
:1065B000129611961C921E92129687E19DE21196F8
:1065C0009C938E93129611961C921E92129683E1C2
:1065D0009DE28D939C93E858FF4F1182108208959D
:1065E00008956E3471050CF050C06B3471050CF0D9
:1065F0008FC06C32710554F5693271050CF088C09A
:106600006831710594F46F3071050CF081C066300B
:10661000710544F4623071050CF07AC0672B09F003
:1066200075C076C06B5071096EC0623271053CF462
:106630006F3171050CF06CC06951710964C064520E
:1066400071096230710508F061C062C06A3371057A
:106650007CF4673371050CF05BC06D3271050CF48E
:1066600055C0603371050CF453C0635371094BC0BE
:10667000643471053CF4613471050CF049C06D530C
:10668000710941C0675471093EC066387105F4F460
:1066900063387105ECF56237710564F46F36710586
:1066A000BCF56536710594F1683671058CF1695653
:1066B000710929C06C37710534F46937710544F5E7
:1066C0006357710920C06D5771091DC0603D710588
:1066D0007CF46D3C7105E4F46439710534F461397E
:1066E0007105B4F46D5871090EC0695C71090BC075
:1066F0006A3D710534F4673D710554F4635D7109B9
:1067000002C06D5D71096330710510F080E008957D
:1067100081E008950C94D4470C94D4470C94D4474A
:106720000C94D4470C94D4470C94D4470C94D4477D
:106730000C94D4470C94D4470C94D4470C94D4476D
:106740008F929F92AF92BF92CF92DF92EF92FF9281
:106750000F931F930E94DF1660E070E046D2892BF2
:10676000D1F40E94DF161F921F9221E02F931F92F7
:106770001F92812C912CA12CB12CC12CD12C7601F3
:1067800097018601B701A6010E94150B0F900F908B
:106790000F900F900F9080E090E01F910F91FF906D
:1067A000EF90DF90CF90BF90AF909F908F90089523
:1067B0008F929F92AF92BF92CF92DF92EF92FF9211
:1067C0000F931F930E94DF1661E070E00ED2892BB9
:1067D000D1F40E94DF161F9221E02F931F921F9287
:1067E0001F92812C912CA12CB12CC12CD12C760183
:1067F00097018601B701A6010E94150B0F900F901B
:106800000F900F900F9080E090E01F910F91FF90FC
:10681000EF90DF90CF90BF90AF909F908F900895B2
:10682000EF92FF920F931F93CF93DF9300D01F92AD
:10683000CDB7DEB7FB0122A133A144A155A1068D3E
:10684000178D29833A834B835C830E9415097C0151
:10685000FC018281938129813A814B815C818F3057
:10686000F7E29F072CF40196F7019383828303C01C
:10687000F70113821282B801C70129833A834B833F
:106880005C83AFDE29813A814B815C818823A1F052
:10689000F801EE0FFF1FEE0FFF1FEA5AF84F20839B
:1068A000318342835383B801C7010E948308B80132
:1068B000C7010E94D20803C085ED94E0A8D6D2D8C3
:1068C0000E94191B80E090E00F900F900F900F90A6
:1068D000DF91CF911F910F91FF90EF9008950F934B
:1068E0001F93CF93DF930E9415098C01C0E0D0E085
:1068F000BE01C80176DE882321F0BE01C8010E94D6
:10690000D2082196C13ED10599F787E496E07FD65B
:106910000E948B180E94951780E090E0DF91CF9144
:106920001F910F9108958BE496E071D685E593E071
:106930006ED60E948B180E94951780E090E0089513
:106940000E948B18FC01148680E090E008958091ED
:10695000A60B9091A70B892BA1F480E790E00E94F1
:106960003F47FC01F9969C0123593F4FDF01D8971F
:106970001C921192E217F307C9F79093A70B80932B
:10698000A60B8091A60B9091A70B08956F927F9212
:106990008F929F92AF92BF92CF92DF92EF92FF922F
:1069A0000F931F93CF93DF93FB01E2A8F3A886A474
:1069B00097A4A0A8B1A8C6A0D7A062A073A0068D76
:1069C000178DC5DFEC019701A301B8010E942D0AC4
:1069D000C501B4010E943E299701A601B801CE016C
:1069E0000E942D0A80E090E0DF91CF911F910F91DE
:1069F000FF90EF90DF90CF90BF90AF909F908F90DF
:106A00007F906F9008950F931F93CF93DF93FB01B7
:106A100002A913A9C68DD78D9ADFA801BE010E94D5
:106A2000960980E090E0DF91CF911F910F9108953A
:106A30001F93CF93DF931F92CDB7DEB7FB0162A9FF
:106A4000168D698384DF6981812F0E94F72880E099
:106A500090E00F90DF91CF911F910895EF92FF92F8
:106A60000F931F93CF93DF93FB01E2A8F3A802A13A
:106A700013A1C68DD78D6BDF9701A801BE010E94BF
:106A80002D0A80E090E0DF91CF911F910F91FF9050
:106A9000EF90089508950895089508950895CF9367
:106AA000DF93EC0188810E94DB2721E0892B09F428
:106AB00020E02C878C810E94DB2721E0892B09F4C0
:106AC00020E02E878E899F890197D1F48A810E94C8
:106AD000DB2721E0892B09F420E02D878E810E949D
:106AE000DB2721E0892B09F420E02F879C858D8509
:106AF000981749F08E85821731F09A878B8703C0EB
:106B00008C858A872B87DF91CF9108950F93FC01A5
:106B10009285908783858187A689B789119721F40B
:106B2000621721F0401711F062874387838588231D
:106B3000D1F0828591110AC08823A9F080899189BA
:106B4000A289B3890197A109B10909C081110BC0BC
:106B500080899189A289B3890196A11DB11D808B7D
:106B6000918BA28BB38B0F910895CF93DF93FC0190
:106B7000A489B589C08DD18D2089318942895389F5
:106B8000A03187E2B80759F01A161B0644F40E9498
:106B90003E4E20E137E240E050E00E94184EDE0118
:106BA0000E943E4EDF91CF910895FC0181E090E07C
:106BB000938F828F1182108215821482108A118A1B
:106BC000128A138A178A168A80E197E2958B848B42
:106BD00012861086148615861686178608950895DF
:106BE000089508950895089508952F923F924F9221
:106BF0005F926F927F928F929F92AF92BF92CF924D
:106C0000DF92EF92FF920F931F93CF93DF93CDB755
:106C1000DEB7A3970FB6F894DEBF0FBECDBF9BA320
:106C20008AA31B010E94291D8AA19BA10E944E1BC1
:106C30008AA19BA10E94582C8AA19BA10E945C2C36
:106C400021E022163104C9F132E02316310409F49F
:106C500066C02114310409F095C0AAA0BBA040E190
:106C6000A40EB11C8AA19BA182589E4F9E838D8346
:106C7000EAA1FBA1EA5BFD4F90819D87AAA1BBA180
:106C8000A959BD4FB887AF83EAA1FBA1EF56FD4FCD
:106C9000F98BE88B2AA13BA12D553D4F3D8B2C8BC9
:106CA0004AA15BA14D515E4F5C874B878DE890E018
:106CB0009B8B8A8BA5E1B0E062C0AAA0BBA0BAE81A
:106CC000AB0EB11CEAA1FBA1E656FE4FFE83ED839D
:106CD000EAA1FBA1E95BFD4F20812D874AA15BA1C1
:106CE00045595D4F58874F838AA19BA18D569D4F73
:106CF000998B888BAAA1BBA1AC55BD4FBD8BAC8B2A
:106D0000EAA1FBA1EB51FE4FFC87EB872EE830E0B8
:106D10003B8B2A8B46E150E05C834B8336C0AAA0B4
:106D2000BBA05CEFA51A5EEFB50A8AA19BA18A54AD
:106D30009E4F9E838D83EAA1FBA1E85BFD4F90816E
:106D40009D87AAA1BBA1A159BD4FB887AF83EAA176
:106D5000FBA1EB56FD4FF98BE88B2AA13BA12B55EC
:106D60003D4F3D8B2C8B4AA15BA149515E4F5C8707
:106D70004B878FE890E09B8B8A8BA7E1B0E0BC83C8
:106D8000AB8303C080E596E00CC0C5010E94B72D1F
:106D9000811105C0C5010E94A72D882369F081EEED
:106DA00096E035D40E948B1881E090E090934507DF
:106DB0008093440790E0C8C384E294E028D48FE72E
:106DC00096E025D4D5018C9163D487E197E01FD458
:106DD0008CE993E01CD481E090E0EB85FC85918305
:106DE000808341E050E0B5018AA19BA10E94E31895
:106DF000C5010E94092ED5019C968C918501005AEF
:106E00001F4F882339F0C5010E94DF2D81E0F80172
:106E1000808305C0C5010E94C72DD8011C928D81B9
:106E20009E81A3DEF501FE96608371838283938346
:106E3000EF81F8851082118212821382EAA1FBA1F0
:106E4000E959FD4F1082118212821382EAA1FBA13F
:106E5000E559FD4F1082118212821382EAA1FBA133
:106E6000E159FD4F108211821282138286E090E078
:106E7000AB85BC858D939C9346E050E0B5018AA11B
:106E80009BA10E94E31841E050E0B5018AA19BA1BB
:106E90000E94C818412C512C320143948AA19BA115
:106EA000820D931DFC01ED55FD4FFF87EE874101DB
:106EB000880C991C880C991CC40189569D4F2AA1E5
:106EC0003BA1280F391F3F8B2E8BC101875A9E4F44
:106ED000880F991F4AA15BA1480F591F5B8F4A8FEA
:106EE000C4018B579D4FAAA1BBA1A80FB91FBD8F8D
:106EF000AC8FF401E758FD4FFF8FEE8F8AA19BA165
:106F0000880D991D9C01205F3D4F3A872987AE85EA
:106F1000BF858C918823B1F0A40149595D4FEAA146
:106F2000FBA14E0F5F1FCE88DF88EA8CFB8C0C8D97
:106F30001D8D2E8D3F8D2E0F3F1F6D817E81C501D2
:106F40000E949C2B88EA9BE00E94E62418161906F2
:106F500024F01A82198210E01DC088EA9BE00E948A
:106F6000C4248F7D85349105A1F782E095E04FD34D
:106F70000E948B1821E0DC011C962C9382E693E0A2
:106F800046D30E948B180E949517E1E0F0E0FA8347
:106F9000E98311E0C5010E94B72D8111C4C2C5016A
:106FA0000E94A72D8111BFC21111BDC2A889B98944
:106FB0006D917C91072E000C880B990B0E94EC4C74
:106FC0009B01AC01EF81F8856081718182819381A1
:106FD0000E94E64C87FFA7C2C5010E94B22EE98538
:106FE000FA85208131814281538160E573EC80E034
:106FF00090E00E94184EC9010E943329A985BA85E4
:107000002D913D914D915C91A3E0B0E00E94344EF2
:107010009B01AC01C301B2010E94184E672B682B83
:10702000692B39F48EE593E0F2D20E948B180E940E
:107030009517C5010E948E2DA985BA852D913D9188
:107040004D915C9160E573EC80E090E00E94184EF9
:10705000C9010E943329BFEF4B1A5B0A6B0A7B0AF6
:10706000E981FA81EF2B09F452CF21E030E03A8335
:10707000298342E050E0B5018AA19BA10E94C81873
:1070800084E294E0C4D28FE796E0C1D2D5018C911E
:10709000FFD286E896E0BBD28CE993E0B8D2E981D2
:1070A000FA81EF2BD1F489E996E0B1D28EE496E033
:1070B000AED281ED94E0ABD28B819C811BD38EE468
:1070C00096E0A5D283ED94E0A2D2FD858F2F90E0CB
:1070D00011D30E948B180E9495178AA19BA10E9430
:1070E000582C8AA19BA10E945C2C84E294E08FD250
:1070F0008FE796E08CD2D5018C91CAD28DE996E0CB
:1071000086D28CE993E083D2EF81F88510821182D8
:1071100012821382D5019C968C918501005A1F4FD3
:10712000882331F0C5010E94C72DF801108206C0E6
:10713000C5010E94DF2D81E0D8018C938D819E8155
:1071400014DDF501FE966083718382839383EAA147
:10715000FBA1E959FD4F1082118212821382EAA12C
:10716000FBA1E559FD4F1082118212821382EAA120
:10717000FBA1E159FD4F10821182128213828D8191
:107180009E81F3DC6E8B7F8B888F998F412C512CE5
:10719000320143948AA19BA1820D931DFC01ED5500
:1071A000FD4FFB8FEA8F9101220F331F220F331FF8
:1071B0003C832B83C90189569D4F4AA15BA1480F8F
:1071C000591F5D8F4C8FC101875A9E4F880F991FA1
:1071D000AAA1BBA1A80FB91FBF8FAE8FC9018B5742
:1071E0009D4FEAA1FBA1E80FF91FF9A3E8A3C9018C
:1071F0002AA13BA1820F931FAC01405F5D4F5F87C7
:107200004E879201215031093A87298749014981E6
:107210005A81452B09F0C7C0AA8DBB8D8C9188235C
:10722000C9F02B813C8127583D4FEAA1FBA12E0FCD
:107230003F1F4B815C8149595D4F4E0F5F1FCC8CC6
:10724000DD8CEE8CFF8C08A119A16D817E81C501BA
:107250000E949C2B88EA9BE00E94E62418161906DF
:1072600014F010E01DC088EA9BE00E94C4248F7DCA
:1072700085349105B1F782E095E0C9D10E948B1861
:1072800021E0DC011C962C9382E693E0C0D10E94A1
:107290008B180E949517E1E0F0E0FA83E98311E092
:1072A00029853A852A30310538F4AF81B8851D9299
:1072B0001D921D921C921397BD85C501B1113FC14E
:1072C0000E94A72D81116BC0112319F089849A8423
:1072D00066C0E889F98960817181072E000C880BEE
:1072E000990B0E94EC4C9B01AC01AF81B8856D916C
:1072F0007D918D919C910E94E64C87FFE7CFC5015F
:107300000E94B22EEE85FF8520813181428153811A
:1073100060E573EC80E090E00E94184EC9010E9485
:107320003329AE85BF852D913D914D915C91A3E0B0
:10733000B0E00E94344E9B01AC01C301B2010E9437
:10734000184E672B682B692B91F48EE593E05FD183
:107350000E948B180E94951784E294E058D181EB2B
:1073600096E055D1C201C6D18CE993E050D1C50158
:107370000E948E2DEE85FF852081318142815381CF
:1073800060E573EC80E090E00E94184EC9010E9415
:107390003329FFEF4F1A5F0A6F0A7F0A32CF8FEB54
:1073A00096E035D104C081E090E09A83898384E23D
:1073B00094E02DD18FE796E02AD1D5018C9168D148
:1073C00083ED96E024D18CE993E021D18D819E81DB
:1073D000CCDBEC89FD89EF2BA1F0DC01CB012E8900
:1073E0003F89488D598D821B930BA40BB50BB7FFBA
:1073F00007C0B095A095909581959F4FAF4FBF4F17
:107400004C0149815A81452BF9F489E996E0FFD076
:107410008EE496E0FCD081ED94E0F9D08A899B89D6
:1074200069D18EE496E0F3D083ED94E0F0D0B4011E
:10743000092C000C880B990B0E94EC4C42E05FD1A8
:107440000E948B180E94951785E090E0AB85BC8563
:107450008D939C9345E050E0B5018AA19BA10E94C9
:10746000E318C5010E94F72D8AA19BA10E94582C08
:107470008AA19BA10E945C2CB1E02B163104A9F0DB
:10748000E2E02E16310401F1232861F50E948B18E9
:10749000C401990CAA0BBB0B80934A0790934B072E
:1074A000A0934C07B0934D071DC00E948B18C401D8
:1074B000990CAA0BBB0B80934E0790934F07A09398
:1074C0005007B09351070EC00E948B18C401990C4D
:1074D000AA0BBB0B8093520790935307A0935407BA
:1074E000B09355070E948B180E94E817AB85BC85A6
:1074F0001D921C9240E050E0B5018AA19BA10E9420
:10750000E31840E050E0B5018AA19BA10E94C81891
:107510000E948B18E981FA81F0934507E0934407B4
:1075200089819A8111C08FEB96E071D0C5010E94CC
:10753000A72D882309F49DCDB1E0BD879ACD0E9487
:10754000B72D8111C3CEC0CEA3960FB6F894DEBF7F
:107550000FBECDBFDF91CF911F910F91FF90EF90A4
:10756000DF90CF90BF90AF909F908F907F906F9063
:107570005F904F903F902F900895CF93DF93FC0141
:10758000EA52FE4F408151814115510559F1EC01FC
:10759000C652DE4F288139818E529E4F24173507FF
:1075A000C8F4FC0180819181009761F0FC01E20F39
:1075B000F31F80818A3041F08D3029F48CE993E00B
:1075C00026D002C080E064D0888199810196998399
:1075D000888308C040E050E06EE973E00E943E27D7
:1075E00019821882DF91CF910895009769F0FC010C
:1075F00001900020E9F73197AF01481B590BBC01FE
:1076000088EA9BE00C94862480E090E00895EDCF1A
:107610008F929F92AF92BF920F931F93CF93DF935E
:10762000CDB7DEB7A1970FB6F894DEBF0FBECDBFC2
:1076300019A2423008F44AE08E010F5D1F4F842EDC
:10764000912CA12CB12CA50194010E94444EE62F4F
:10765000B901CA0101501109EA3014F4E05D01C01A
:10766000E95CD801EC93232B242B252B61F7C8016F
:10767000BCDFA1960FB6F894DEBF0FBECDBFDF9181
:10768000CF911F910F91BF90AF909F908F900895D1
:10769000E091A80BF091A90B0190F081E02D682FEB
:1076A00088EA9BE01994CF92DF92EF92FF92CF93FA
:1076B000DF9397FF17C06B017C018DE2E9DFEC01DE
:1076C00066277727CB016C197D098E099F094AE04F
:1076D0009FDF8C0F9D1FDF91CF91FF90EF90DF9088
:1076E000CF9008954AE0DF91CF91FF90EF90DF9027
:1076F000CF908ECFBC01990F880B990BD4CF4F92AE
:107700005F926F927F928F929F92AF92BF92CF9231
:10771000DF92EF92FF926B017C01B42E9B01AC01D2
:107720000E94774F882319F086E397E027C026014F
:107730003701E89477F82FEF3FEF4FE75FE7C3019A
:10774000B2010E94774F81110DC02FEF3FEF4FE73D
:107750005FE7C301B2010E94E64C18161CF48AE3ED
:1077600097E00CC02FEF3FEF4FE75FE4C701B60192
:107770000E94734F18167CF48EE397E0FF90EF9011
:10778000DF90CF90BF90AF909F908F907F906F9041
:107790005F904F902ACF2FEF3FEF4FE75FECC7018D
:1077A000B6010E94E64C87FDE7CF20E030E0A9015A
:1077B000C701B6010E94E64C87FF08C08DE268DF72
:1077C0004C01F7FAF094F7F8F09402C0812C912C58
:1077D000A12C60E070E080E09FE3AB1441F020E07A
:1077E00030E040E251E40E94DA4EA394F6CF9B01D0
:1077F000AC01C701B6010E94764E2B013C010E94EC
:10780000474F6B017C010E94EA4C9B01AC01C30114
:10781000B2010E94754E2B013C014AE0C701B6013E
:10782000F7DE7C01E80CF91CBB2021F08EE230DF92
:10783000E80EF91EDB2CDD2019F120E030E040E2FB
:1078400051E4C301B2010E944B4D2B013C010E9447
:10785000474F4B01A12CB12C4AE0C501B401D8DE41
:10786000E80EF91EC501B4010E94EA4C9B01AC016F
:10787000C301B2010E94754E2B013C01DA94DBCFAB
:10788000C701FF90EF90DF90CF90BF90AF909F9097
:107890008F907F906F905F904F900895789484B50B
:1078A000826084BD84B5816084BD85B5826085BDFC
:1078B00085B5816085BD80916E00816080936E008A
:1078C000109281008091810082608093810080917C
:1078D000810081608093810080918000816080932D
:1078E00080008091B10084608093B1008091B000ED
:1078F00081608093B00080919100826080939100BC
:1079000080919100816080939100809190008160CE
:10791000809390008091A10082608093A10080916B
:10792000A10081608093A1008091A000816080937C
:10793000A00080912101826080932101809121012A
:1079400081608093210180912001816080932001DA
:1079500080917A00846080937A0080917A008260BE
:1079600080937A0080917A00816080937A00809180
:107970007A00806880937A001092C10061E086E30B
:107980000E94F72861E087E30E94F72861E086E221
:107990000E94F72861E08AE10E94F72861E08CE10B
:1079A0000E94F72861E088E10E94F72862E083E006
:1079B0000E94F72862E082E00E94F72862E080E1FE
:1079C0000E94F72862E081E10E94F72862E08FE1DF
:1079D0000E94F72862E081E20E94F72861E08CE3D0
:1079E0000E94F72861E08DE30E94F72861E088E3B8
:1079F0000E94F72862E08EE00E94F72862E08FE0A4
:107A00000E94F72862E087E10E94F72862E089E19E
:107A10000E94F72862E083E20E94F72862E085E294
:107A20000E94F72861E08EE20E94F72861E080E37F
:107A30000E94F72861E08EE30E94F72862E082E16D
:107A40000E94F72862E083E10E94F72862E08BE160
:107A50000E94F72862E08DE10E94F72862E087E249
:107A60000E94F72862E089E20E94F72861E08AE03C
:107A70000E94F72861E088E00E94F72861E089E031
:107A80000E94F72861E08DE00E94F72862E08FE312
:107A90000E94F72862E08BE30E94F72862E088E208
:107AA0000E94F72862E080E40E94F72862E08AE200
:107AB0000E94F72862E08CE20E94F72862E081E4ED
:107AC0000E94F72862E082E40E94F72862E084E3E3
:107AD0000E94F72862E085E30E94F72862E080E0D8
:107AE0000E94F72862E081E00E94F72862E089E3C3
:107AF0000E94F72862E08AE30E94F72862E081E3AF
:107B00000E94F72862E082E30E94F72862E083E3A4
:107B10000E94F72862E08BE20E94F72862E08DE283
:107B20000E94F72862E08FE20E94F72862E080E27C
:107B30000E94F72861E086E20E94032861E088E164
:107B40000E94032861E088E30E94032861E08EE33D
:107B50000E940328E091B80BF091B90B82E080837A
:107B6000E091B40BF091B50B1082E091B60BF0915F
:107B7000B70BD0E1D0831092C00BE091BC0BF09119
:107B8000BD0B86E08083E091BA0BF091BB0B808146
:107B900080618083E091BA0BF091BB0B808188609B
:107BA0008083E091BA0BF091BB0B80818068808369
:107BB000E091BA0BF091BB0B80818F7D808364E6EE
:107BC00070E080E090E00E943E290E94DF160E9453
:107BD00087130E94322D0E94191B0E947629609300
:107BE0007E0B70937F0B8093800B9093810B82EDC3
:107BF00097E09093430780934207C1E0C0936F00E2
:107C0000D093810010928000C093DC0A80E092E063
:107C10009093DB0A8093DA0A909387008093860022
:107C200081E1809381001092810010928500109272
:107C300084008091DC0A8061809381000E94762913
:107C400060937A0B70937B0B80937C0B90937D0BEE
:107C50000E9476296093820B7093830B8093840B30
:107C60009093850B0E94762960937E0B70937F0B17
:107C70008093800B9093810B0E94150980915E0781
:107C800090915F07A0916007B09161070197A105EE
:107C9000B10579F40E9415098091A6079091A70774
:107CA000A091A807B091A9070197A105B10509F412
:107CB000C9C70E94150980915E0790915F07A09146
:107CC0006007B09161070197A105B10579F40E94A1
:107CD00015098091A2079091A307A091A407B091E4
:107CE000A5070197A105B10509F4CAC70E941509A6
:107CF00080915E0790915F07A0916007B091610746
:107D00000197A105B10579F40E94150980919E079C
:107D100090919F07A091A007B091A1070197A1059D
:107D2000B10509F4CCC780E893E071DC8FE7282E19
:107D300082E0382E95E7A92E92E0B92E0E9476298E
:107D40006093820B7093830B8093840B9093850BCD
:107D500000917E0B10917F0B2091800B3091810B55
:107D6000601771078207930748F460937E0B709346
:107D70007F0B8093800B9093810B2CC0DC01CB0197
:107D8000801B910BA20BB30B883E9340A105B1055C
:107D900008F108511C4F2F4F3F4F00937E0B10935B
:107DA0007F0B2093800B3093810B0E94322DEC01CE
:107DB0000E94042BCE010C960E94042BCE01489603
:107DC0000E94042BCE0184960E94042BCE01C09603
:107DD0000E94042B88EA9BE00E94E624892B09F488
:107DE000BCC50E94762960937A0B70937B0B8093BD
:107DF0007C0B90937D0B88EA9BE00E94C4248093C7
:107E0000790B982F9F7D953479F02091770B3091E5
:107E1000780BF901EB5BF44F80832F5F3F4F30937A
:107E2000780B2093770B06C00E948B1821E0DC01B1
:107E30001C962C938091770B9091780B8133910550
:107E400064F02AE02093790BFC01EB5BF44F208374
:107E500001969093780B8093770B8091790B20910A
:107E6000770B3091780B8A3039F4C9010197A2E180
:107E7000BBE0E5E4FBE004C022333105B4F76DC597
:107E8000AF0145545B40481759071CF441914D938D
:107E9000F7CFFC01EE5EF44F1082223031050CF476
:107EA00058C581E193E0B3DB8EE496E0B0DB8FE967
:107EB00093E0ADDB82E19BE0AADB8FE993E0A7DBF7
:107EC0008CE993E0A4DB8AE390E0D9D7EC011A8235
:107ED0001B821C821D821E821F82188619861A86AA
:107EE0001B861C861D861E861F86188A198A1A8A7A
:107EF0001B8A1C8A1D8A1E8A1F8A188E198E1A8E4A
:107F00001B8E1C8E1D8E1E8E1F8E18A219A21AA2E9
:107F10001BA21CA21DA21EA21FA218A619A61AA669
:107F20001BA61CA61DA61EA61FA618AA19AA1AAA39
:107F30001BAA1CAA1DAA1EAA1FAA18AE19AE68E089
:107F400072E082E19BE00E946F488C01FC0180811D
:107F50008654823008F027C161EA73E0C8010E94AC
:107F60007750892B09F4D3C064EA73E0C8010E94FA
:107F70007750892B09F4CBC068EA73E0C8010E94EE
:107F80007750892B09F4C6C06BEA73E0C8010E94E0
:107F90007750892B09F4BEC06FEA73E0C8010E94D4
:107FA0007750892B09F4B9C063EB73E0C8010E94D4
:107FB0007750892B09F4B4C067EB73E0C8010E94C5
:107FC0007750892B09F4ACC06AEB73E0C8010E94BA
:107FD0007750892B09F4A7C06EEB73E0C8010E94AB
:107FE0007750892B09F4A2C062EC73E0C8010E94AB
:107FF0007750892B09F49DC066EC73E0C8010E949C
:108000007750892B09F498C06AEC73E0C8010E948C
:108010007750892B09F493C06EEC73E0C8010E947D
:108020007750892B09F48EC062ED73E0C8010E947D
:108030007750892B09F489C066ED73E0C8010E946E
:108040007750892B09F484C06AED73E0C8010E945F
:108050007750892B09F47FC06EED73E0C8010E9450
:108060007750892B09F47AC062EE73E0C8010E9450
:108070007750892B09F475C066EE73E0C8010E9441
:108080007750892B09F470C06AEE73E0C8010E9432
:108090007750892B09F46BC06EEE73E0C8010E9423
:1080A0007750892B09F466C062EF73E0C8010E9423
:1080B0007750892B09F461C066EF73E0C8010E9414
:1080C0007750892B09F45CC06AEF73E0C8010E9405
:1080D0007750892B09F457C06EEF73E0C8010E94F6
:1080E0007750892B09F452C062E074E0C8010E9405
:1080F0007750892B09F44DC066E074E0C8010E94F6
:108100007750892B09F448C08FEF9FEF47C080E07C
:1081100090E044C081E090E041C08CE190E03EC03E
:108120008DE690E03BC08FE690E038C080E790E0BD
:1081300035C081E790E032C082E790E02FC083E74E
:1081400090E02CC084E790E029C088E790E026C04A
:1081500089E790E023C08AE790E020C083E890E0C0
:108160001DC084E890E01AC08DE890E017C08EE84A
:1081700090E014C08FE890E011C080E990E00EC05C
:1081800081EA90E00BC085EB90E008C086EB90E0C0
:1081900005C087EB90E002C088EB90E0909301026D
:1081A00080930002BBC08FEF9FEF909301028093FA
:1081B0000002B8C0D8018C91883539F4C801019605
:1081C0008BD76A837B838C839D83F801808189357B
:1081D00039F4C801019680D76E837F838887998799
:1081E000D8018C918A3539F4C801019675D76A8710
:1081F0007B878C879D87F8018081813449F4C80191
:1082000001966AD70E94424F6E877F87888B998B31
:10821000D8018C91823449F4C80101965DD70E943F
:10822000424F6A8B7B8B8C8B9D8BF80180818334D2
:1082300049F4C801019650D70E94424F6E8B7F8B44
:10824000888F998FD8018C91833539F4C8010196B4
:1082500043D76A8F7B8F8C8F9D8FF801808180350B
:1082600049F4C801019638D70E94424F6E8F7F8F24
:1082700088A399A3D8018C91863549F4C801019649
:108280002BD70E94424F6AA37BA38CA39DA3F80126
:108290008081873549F4C80101961ED70E94424F5C
:1082A0006EA37FA388A799A7D8018C91853449F440
:1082B000C801019611D70E94424F6AA77BA78CA7DD
:1082C0009DA7F8018081843549F4C801019604D73F
:1082D0000E94424F6EA77FA788AB99ABD8018C91C3
:1082E0008D3449F4C8010196F7D60E94424F6AAB1B
:1082F0007BAB8CAB9DABF8018081813549F4C80123
:108300000196EAD60E94424F6EAB7FAB88AF99AF21
:108310006AE074E080E090E0E2D68C01011511057E
:1083200009F048CF0E948B18DC011C961C910E941A
:10833000150940906A0750906B0760906C07709029
:108340006D07CEA8DFA8E8ACF9AC0E948B18C092EC
:108350004607D0924707E0924807F092490780917C
:10836000000290910102992493948230910538F093
:108370009C012F5631092630310508F0912C11232C
:1083800071F08D36910559F09C0128573109233041
:10839000310528F0855B9109039708F0D0C20E944F
:1083A000150980915E0790915F07A0916007B091D9
:1083B00061070197A105B10529F0992019F08DEF0A
:1083C00092E0BFC2209719F489EF92E0BAC2E09020
:1083D0000002F0900102BFEFEB16FB06A9F3E114D7
:1083E000F104B9F48091DD0A9091DE0A892B61F4E1
:1083F00082E090E044D521E132E0FC01318320832A
:108400009093DE0A8093DD0A0091DD0A1091DE0A66
:108410006EC0FCE1EF16F104B9F48091DF0A90918F
:10842000E00A892B61F482E090E029D52BE132E06B
:10843000DC012D933C939093E00A8093DF0A009136
:10844000DF0A1091E00A53C0BDE6EB16F104B9F45F
:108450008091E10A9091E20A892B61F482E090E038
:108460000ED525E232E0FC01318320839093E20AAD
:108470008093E10A0091E10A1091E20A53C0FFE6FD
:10848000EF16F104B9F48091E30A9091E40A892B84
:1084900061F482E090E0F3D42FE232E0DC012D932E
:1084A0003C939093E40A8093E30A0091E30A1091CD
:1084B000E40A53C000E010E0B0E7EB16F104B9F4B1
:1084C0008091E50A9091E60A892B61F482E090E0C0
:1084D000D6D429E332E0FC01318320839093E60A6D
:1084E0008093E50A0091E50A1091E60A6CC0F1E775
:1084F000EF16F104B9F48091E70A9091E80A892B0C
:1085000061F482E090E0BBD423E432E0DC012D93FF
:108510003C939093E80A8093E70A0091E70A109150
:10852000E80A6CC0B2E7EB16F104B9F48091E90AED
:108530009091EA0A892B61F482E090E0A0D42DE4C6
:1085400032E0FC01318320839093EA0A8093E90AA8
:108550000091E90A1091EA0A6AC0F3E7EF16F10404
:10856000B9F48091EB0A9091EC0A892B61F482E0D6
:1085700090E085D427E532E0DC012D933C93909385
:10858000EC0A8093EB0A0091EB0A1091EC0A68C0A8
:10859000B4E7EB16F104B9F48091ED0A9091EE0A7C
:1085A000892B61F482E090E06AD421E632E0FC019C
:1085B000318320839093EE0A8093ED0A0091ED0AB7
:1085C0001091EE0A68C0F8E7EF16F104B9F4809153
:1085D000EF0A9091F00A892B61F482E090E04FD489
:1085E0002BE632E0DC012D933C939093F00A8093CC
:1085F000EF0A0091EF0A1091F00A68C0B9E7EB1694
:10860000F104A9F48091F10A9091F20A892B51F4B6
:1086100082E090E034D4FC01B182A0829093F20A0F
:108620008093F10A0091F10A1091F20A6AC0FAE708
:10863000EF16F104A9F48091F30A9091F40A892BC2
:1086400051F482E090E01BD4DC012D923C92909397
:10865000F40A8093F30A0091F30A1091F40A6CC0B3
:10866000BDE8EB16F104B9F48091F50A9091F60A91
:10867000892B61F482E090E002D429E832E0FC0129
:10868000318320839093F60A8093F50A0091F50ACE
:108690001091F60A6CC03EE8E316F104B9F480913B
:1086A000F70A9091F80A892B61F482E090E0E7D311
:1086B000E3E9F2E0DC01ED93FC939093F80A8093F8
:1086C000F70A0091F70A1091F80A6CC0FFE8EF165C
:1086D000F104B9F48091F90A9091FA0A892B61F4B6
:1086E00082E090E0CCD3EDE9F2E0DC01ED93FC9385
:1086F0009093FA0A8093F90A0091F90A1091FA0A04
:108700006CC0F0E9EF16F104B9F48091FB0A909186
:10871000FC0A892B61F482E090E0B1D3E7EAF2E051
:10872000DC01ED93FC939093FC0A8093FB0A00918B
:10873000FB0A1091FC0A6CC0F1EAEF16F104B9F4DF
:108740008091FD0A9091FE0A892B61F482E090E00D
:1087500096D3E1EBF2E0DC01ED93FC939093FE0AFB
:108760008093FD0A0091FD0A1091FE0A6BC0F5EBA3
:10877000EF16F104B9F48091FF0A9091000B892B58
:1087800061F482E090E07BD3EBEBF2E0DC01ED936F
:10879000FC939093000B8093FF0A0091FF0A1091C5
:1087A000000B50C0F6EBEF16F104B9F48091010B09
:1087B0009091020B892B61F482E090E060D3E5ECAC
:1087C000F2E0DC01ED93FC939093020B8093010B9C
:1087D0000091010B1091020B35C0F7EBEF16F1047D
:1087E000B9F48091030B9091040B892B61F482E022
:1087F00090E045D3EFECF2E0DC01ED93FC93909335
:10880000040B8093030B0091030B1091040B1AC00F
:10881000F8EBEF16F104B1F48091050B9091060B83
:10882000892B61F482E090E02AD3E3EEF2E0DC01F0
:10883000ED93FC939093060B8093050B0091050B31
:108840001091060B0115110589F489EF92E00E9441
:10885000073B0E948B180E9495178EE094E00E94BF
:10886000F53A8CE993E00E94F53A71C085EF92E009
:108870000E94073B0E948B180E9495170E948B183C
:108880001092450710924407E12CF12CFFEFEF1AEC
:10889000FF0A21E0E216F10441F081EF92E00E942C
:1088A000073B0E948B180E949517D801ED91FC910F
:1088B0000480F581E02DBE01C80119950E948B1836
:1088C000C0904407D09045070E948B18FC01848516
:1088D000E114F104D9F281110AC0E414F5043CF466
:1088E000C114D10421F0F2E0CF16D10479F688EA60
:1088F0009BE00E94E624181619062CF488EA9BE0F7
:108900000E94C424F4CFCD2809F4FBC1992009F4B6
:10891000F5C10E9415098091660790916707A091A3
:108920006807B09169070197A105B10509F0E6C193
:108930000E948B1821E0DC011C962C93DFC181E0A2
:1089400093E00E94073B0E948B180E949517CE016E
:108950002BD31092780B1092770B8091110B811111
:1089600070C00E948B18FC018485882309F469C0BB
:108970000E94DF16EC01FC01EE53FD4F1082409681
:108980000E94F72DCE0186579F4F0E94F72DCE01F2
:108990008C5F9E4F0E94F72D0E94A7347C018C01B2
:1089A000075C1F4FC1E0D0E06801F8E3CF1AD1089F
:1089B000D6018C918823D9F084E294E00E94073B91
:1089C00088E294E00E94073BCE010E947A3B8CE94A
:1089D00093E00E94073B60E08C2F0E94032840E058
:1089E00050E0BE01C7010E949609F6011082D8012D
:1089F0008C918823F9F084E294E00E94073B8FE396
:108A000094E00E94073BCE010E947A3B8CE993E000
:108A10000E94073B61E08C2F0E94F72860E08C2FBA
:108A20000E94032841E050E0BE01C7010E94960960
:108A3000F801108221960F5F1F4FC533D10509F051
:108A4000B3CF0E948B18DC011C968C918093110B84
:108A5000C0910F0BD091100B0E941509FC0182816F
:108A60009381C817D90799F00E941509DC01129665
:108A70008D919C9113979093100B80930F0B0E94F4
:108A8000DF160E9487130E94322D0E94191B0E943C
:108A9000762960930B0B70930C0B80930D0B9093C6
:108AA0000E0B00917A0B10917B0B20917C0B309177
:108AB0007D0B601771078207930708F4B6C0DC01CD
:108AC000CB01801B910BA20BB30B89389341A105FD
:108AD000B10508F4B4C00E948B18DC011C968C917F
:108AE000882319F08DE093E002C089E093E00E94B2
:108AF000073B0E948B180E9495170E94DF16EC011D
:108B0000FC01ED55FD4F8081882341F0CE01825854
:108B10009E4F0E94B5356B017C0107C0FE01E25BF0
:108B2000FF4FC080D180E280F3800E948B18C092FA
:108B30004A07D0924B07E0924C07F0924D07FE0196
:108B4000EC55FD4F8081882341F0CE0186569E4F23
:108B50000E94B5356B017C0107C0FE01E853FF4F51
:108B6000C080D180E280F3800E948B18C0924E07B3
:108B7000D0924F07E0925007F0925107FE01EB555B
:108B8000FD4F8081882341F0CE018A549E4F0E9480
:108B9000B5356B017C0106C0CE5BDE4FC880D98045
:108BA000EA80FB800E948B18C0925207D092530734
:108BB000E0925407F09255070E948B180E94E81724
:108BC0000E94DF160E9472190E948B180E94D21A0E
:108BD0000E948B180E94A7170E94150980915E07BA
:108BE00090915F07A0916007B09161070197A1057F
:108BF000B10541F085E093E00E94073B0E948B188D
:108C00000E9495178091070B9091080BA091090B7A
:108C1000B0910A0B0196A11DB11D8093070B909393
:108C2000080BA093090BB0930A0B0E94762960935E
:108C30007A0B70937B0B80937C0B90937D0B0E943F
:108C400083257CC885E594E00E94073B0E94DF16DF
:108C5000CF931F921F921F921F92812C912CA12CB7
:108C6000B12CC12CD12C760197018601B701A60148
:108C70000E94150B0F900F900F900F900F9019C836
:108C80008DE694E00E94073B0E94DF161F9221E0D0
:108C90002F931F921F921F92812C912CA12CB12CEB
:108CA000C12CD12C760197018601B701A6010E9443
:108CB000150B0F900F900F900F900F9017C885E82D
:108CC00094E00E94073B0E94DF161F921F9221E052
:108CD0002F931F921F92812C912CA12CB12CC12C6F
:108CE000D12C760197018601B701A6010E94150BD0
:108CF0000F900F900F900F900F9015C889EE92E093
:108D000002C08DEE92E00E94073B0E948B180E94E9
:108D100095170E948B1810924607109247071092E1
:108D200048071092490713CE8091450C9091460C4C
:108D30003BC11092AB0B1092AA0B88EE93E0A0E01F
:108D4000B0E08093AC0B9093AD0BA093AE0BB093BF
:108D5000AF0B8AE693E09093A90B8093A80B85EC68
:108D600090E09093B50B8093B40B84EC90E09093DB
:108D7000B70B8093B60B80EC90E09093B90B809387
:108D8000B80B81EC90E09093BB0B8093BA0B82EC14
:108D900090E09093BD0B8093BC0B86EC90E0909399
:108DA000BF0B8093BE0B1092C10B1092C20B10929E
:108DB000C30B1092C40B82E090E061D02CE733E04B
:108DC000FC013183208390934C0C80934B0C6EE913
:108DD00073E085E49CE00E9468278091DD0C80337D
:108DE00020F09FEF9093DE0C11C08093DE0C282FB3
:108DF00030E0F901EE0FFF1F2E0F3F1FF901E35B7B
:108E0000F34F28EB3BE0328321838F5F803390F474
:108E10008093E10C282F30E0F901EE0FFF1F2E0F99
:108E20003F1FF901E35BF34F28EB3BE032832183E3
:108E30008F5F03C09FEF9093E10C8093DD0C08954A
:108E4000EF920F931F93CF93DF93E80147FD02C08A
:108E500034E001C034E1E42F440FFF0BF7FF03C0FF
:108E6000F195E195F109E32E022F2E2FAE01B3D13A
:108E7000CE01DF91CF911F910F91EF900895CF9385
:108E8000DF938230910510F482E090E0E091E80CED
:108E9000F091E90C20E030E0C0E0D0E0309711F133
:108EA0004081518148175907C0F04817590761F4AC
:108EB00082819381209719F09B838A832BC09093A2
:108EC000E90C8093E80C26C02115310519F04217F2
:108ED000530718F49A01BE01DF01EF010280F3810C
:108EE000E02DDCCF2115310509F1281B390B243089
:108EF000310590F412968D919C911397611571052F
:108F000021F0FB019383828304C09093E90C80934A
:108F1000E80CFD01329644C0FD01E20FF31F81937E
:108F20009193225031092D933C933AC02091E60C45
:108F30003091E70C232B41F420910402309105027B
:108F40003093E70C2093E60C20910202309103024B
:108F50002115310541F42DB73EB7409106025091DD
:108F60000702241B350BE091E60CF091E70CE217A9
:108F7000F307A0F42E1B3F0B2817390778F0AC013C
:108F80004E5F5F4F2417350748F04E0F5F1F509319
:108F9000E70C4093E60C8193919302C0E0E0F0E08F
:108FA000CF01DF91CF9108950F931F93CF93DF935C
:108FB000009709F48CC0FC01329713821282009151
:108FC000E80C1091E90C0115110581F42081318123
:108FD000820F931F2091E60C3091E70C2817390778
:108FE00079F5F093E70CE093E60C71C0D80140E00E
:108FF00050E0AE17BF0750F412962D913C91139795
:10900000AD012115310509F1D901F3CF9D01DA0137
:109010003383228360817181860F971F82179307A4
:1090200069F4EC0128813981260F371F2E5F3F4FED
:10903000318320838A819B8193838283452B29F40A
:10904000F093E90CE093E80C42C01396FC93EE9386
:109050001297ED01499159919E01240F351FE21796
:10906000F30771F480819181840F951F0296119608
:109070009C938E938281938113969C938E931297E7
:10908000E0E0F0E0D80112968D919C911397009743
:1090900019F0F8018C01F6CF8D919C9198012E5F0B
:1090A0003F4F820F931F2091E60C3091E70C281759
:1090B000390769F4309729F41092E90C1092E80C02
:1090C00002C0138212821093E70C0093E60CDF912A
:1090D000CF911F910F9108956627772709C244EE1B
:1090E0005CE000C0FA01A191B081009719F41097DB
:1090F000E1F0CD01DC01CD010D90002011F4C001A3
:1091000013C0FB012191222319F02015D9F7F3CFC9
:10911000FB012191201519F41E92119606C02223FD
:10912000C1F70D900020A1F7D001FA01A193B083FF
:109130000895BB274A3031F4992322F4BDE290957B
:1091400081959F4F30C0BB272A3051F4992342F4B8
:10915000BDE290958095709561957F4F8F4F9F4FA1
:1091600001C0BB27FA01A62F621771058105910581
:10917000330B30FB66F0AA27660F771F881F991FF5
:10918000AA1FA21710F0A21B63953850A9F7A05D83
:10919000AA3308F0A95DA19336F7B111B1931082FB
:1091A000CA0104C4BB27FB015527AA27880F991FB2
:1091B000AA1FA41710F0A41B83955051B9F7A05D06
:1091C000AA3308F0A95DA193009779F7B111B19383
:1091D0001192CB01EBC34F925F926F927F929F925D
:1091E000AF92BF92CF92DF92EF92FF920F931F93B5
:1091F000CF93DF93CDB7DEB729970FB6F894DEBFD4
:109200000FBECDBF6A01122FB02E2BE3201720F026
:10921000FF24F394F00E02C0BCE3FB2E0F2D27E0D9
:10922000AE014F5F5F4FCAD2AC018981982F997010
:10923000913031F0E1FC06C0E0FE06C090E205C0CE
:109240009DE203C09BE201C090E0EE2DE07183FF40
:109250003CC0911102C083E001C084E0811718F482
:10926000212F281B01C020E0E1110BC0F601822F45
:1092700030E2882319F031938150FBCFC20ED11C0C
:1092800020E0992329F0D6019C93F60131966F01D5
:10929000C6010396E2FE0AC03EE4D6013C9341E4D7
:1092A00011964C93119712963C9306C03EE6F60138
:1092B000308341E641833283FC01322F40E2332385
:1092C00009F442C041933150FACF82FF44C091115A
:1092D00002C083E001C084E0811718F4212F281B0D
:1092E00001C020E0E1110BC0F601822F30E288239B
:1092F00019F031938150FBCFC20ED11C20E099238D
:1093000029F0D6019C93F60131966F01C6010396B0
:10931000E2FE0BC039E4D6013C933EE411963C9347
:10932000119736E412963C9307C039E6F601308374
:109330003EE6318336E63283FC01322F40E23323AE
:1093400019F041933150FBCFFC01E20FF11D108267
:109350008EEF9FEFB7C0F1E0911101C0F0E06F2FE9
:1093600070E01416150624F49A012F5F3F4F02C0D7
:1093700021E030E0260F371FBB2029F06B2D70E075
:109380006F5F7F4F02C060E070E0260F371F612FD4
:1093900070E0261737071CF4121B212F01C020E0B4
:1093A0003E2D387159F4D601322F60E2332319F083
:1093B0006D933150FBCFC20ED11C20E0FF2331F062
:1093C000D6019C93B6016F5F7F4F6B01E1110BC01B
:1093D000F601922F30E3992319F031939150FBCF8E
:1093E000C20ED11C20E09F2D940F3A81782F70710E
:1093F000A72E84FF03C0313309F49150191624F4C9
:10940000993018F098E001C091E0E42F852F57FFC4
:1094100002C0E0E080E06E2F782FE0E0F0E0AEE206
:109420009A2E3A01691A71082A01461A570A0B2D19
:1094300010E01195019511096F3F8FEF780729F41E
:10944000D6019C92C60101966C014617570784F01D
:10945000661677066CF47F01E40CF51CA1E0B0E021
:10946000AC0FBD1FEA0EFB1ED7011196BC9002C0C7
:1094700090E3B92E615071093196C60101967C01C5
:109480006017710724F0D601BC926C01D5CF641728
:10949000750741F4363320F4353321F4A11002C0AE
:1094A00081E3B82EF601B082F701822F90E2882383
:1094B00019F091938150FBCFF701E20FF11D10825B
:1094C00080E090E029960FB6F894DEBF0FBECDBFC6
:1094D000DF91CF911F910F91FF90EF90DF90CF9090
:1094E000BF90AF909F907F906F905F904F90089546
:1094F0006F927F928F929F92AF92BF92CF92DF92A4
:10950000EF92FF920F931F93CF93DF93EC017B01B8
:109510006115710519F0DB018D939C938E010F5F2E
:109520001F4F7880872D90E021D2892B11F0E80120
:10953000F5CFBDE27B1205C00F5F1F4F7980C1E000
:1095400008C0EBE27E1204C08E010E5F1F4F7980CF
:10955000C0E06801F1E0CF1AD10843E050E064EFC9
:1095600072E0C6010BD2892BE9F4680122E0C20E39
:10957000D11C45E050E06FEE72E0C601FFD1892BAF
:1095800021F4680187E0C80ED11CE114F10419F040
:10959000D701CD92DC92C111F9C060E070E080E8A3
:1095A0009FE7FDC043E050E06CEE72E0C601E6D1FB
:1095B000892B51F4E114F10409F4EDC00E5F1F4F43
:1095C000F70111830083E7C0680160E070E0CB0120
:1095D00000E010E0F601D0EDD70DDA3050F52C2F79
:1095E0002260622E2C2F2870C2FF05C0211127C0D7
:1095F0000F5F1F4F24C0222311F001501109A5E075
:10960000B0E09B01AC0130D34B015C01880C991C8C
:10961000AA1CBB1CC501B4016D0F711D811D911DDC
:109620006839A9E97A078A07A9E19A0740F0C66074
:1096300005C0DE3F51F4C3FD44C0C8606C2EBFEFCF
:10964000CB1ADB0A7080C62DC5CF2D2F2F7D25317B
:10965000C1F540814D3211F4C06106C04B3221F09A
:10966000319621E030E006C03296D60111964C9139
:1096700022E030E0A0EDA40FAA3018F0E21BF30BBB
:1096800020C040E050E04038BCE05B075CF49A0149
:10969000220F331F220F331F420F531F440F551F3A
:1096A0004A0F511D3196DF0111972C91A0EDA20FA9
:1096B000AA3048F3C4FF03C0519541955109040FE6
:1096C000151FC1FF07C0E114F10421F03197D70144
:1096D000ED93FC937FD1C370C33019F06B017C0113
:1096E00006C06B017C01F7FAF094F7F8F09420E0E3
:1096F00030E0A901C701B60169D1882309F443C04C
:1097000017FF06C0119501951109CBE0D3E002C007
:10971000C3E2D3E05E01B8E1AB1AB1084601BE2D49
:10972000AF2D90E2E92EF12C0E151F057CF0FE0105
:109730002591359145915491B4018B2F9A2FABD13E
:109740004B01B82FA92F0E191F09EECF2497F594BE
:10975000E794CA15DB0541F76401EB2EFA2E8E2D36
:10976000880F8F2D881F8F3F41F020E030E0A90146
:10977000C701B6012BD1811106C082E290E090931F
:10978000EB0C8093EA0CC701B60109C060E070E001
:1097900080E89FEF04C060E070E080EC9FE7DF911D
:1097A000CF911F910F91FF90EF90DF90CF90BF90DE
:1097B000AF909F908F907F906F900895283008F021
:1097C00027E03327DA01990F311D87FD916000965C
:1097D0006105710539F432602E5F3D9330E32A95BF
:1097E000E1F708959F3F30F080387105610509F079
:1097F0003C5F3C5F3D93913008F08068911DDF93A2
:10980000CF931F930F93FF92EF92192F987F969506
:10981000E92F96959695E90FFF27EF57FC4F99276B
:109820003327EE24FF24A701E7010590089407944D
:1098300028F4360FE71EF81E491F511D660F771FCB
:10984000881F991F0694A1F70590079428F4E70E46
:10985000F81E491F561FC11D770F881F991F661FCD
:109860000694A1F70590079428F4F80E491F561F97
:10987000C71FD11D880F991F661F771F0694A1F778
:109880000590079420F4490F561FC71FD81F990F42
:10989000661F771F881F0694A9F78491109517708B
:1098A00041F0D695C79557954795F794E7941A9543
:1098B000C1F7E7E2F3E06894159015913591659151
:1098C000959105907FE27395E118F10A430B560BD1
:1098D000C90BD009C0F7E10CF11E431F561FC91F69
:1098E000D01D7EF4703311F48A95E6CFE8940150D0
:1098F00030F0080F0AF40027021708F4202F2395F0
:10990000022F7A3328F079E37D932A95E9F710C086
:109910007D932A9589F606949795679537951795BF
:109920001794E118F10A430B560BC90BD00998F0B4
:1099300023957E9173957A3308F070E37C9320131E
:10994000B8F77E9170617D9330F0839571E37D93DC
:1099500070E32A95E1F71124EF90FF900F911F918A
:10996000CF91DF91992787FD909508959111F6C0C9
:10997000803219F089508550D0F70895FB01DC0141
:109980004150504088F08D9181341CF08B350CF49F
:10999000805E659161341CF06B350CF4605E861B53
:1099A000611171F3990B0895881BFCCFDC01FC0158
:1099B000672F71917723E1F7329704C07C916D9303
:1099C00070836291AE17BF07C8F3089540D008F4C2
:1099D00081E00895E89409C097FB3EF49095809546
:1099E000709561957F4F8F4F9F4F9923A9F0F92F65
:1099F00096E9BB279395F695879577956795B795E3
:109A0000F111F8CFFAF4BB0F11F460FF1BC06F5FC8
:109A10007F4F8F4F9F4F16C0882311F096E911C0DA
:109A2000772321F09EE8872F762F05C0662371F0FB
:109A300096E8862F70E060E02AF09A95660F771F0F
:109A4000881FDAF7880F9695879597F90895990FEB
:109A50000008550FAA0BE0E8FEEF16161706E807F8
:109A6000F907C0F012161306E407F50798F0621B19
:109A7000730B840B950B39F40A2661F0232B242BEE
:109A8000252B21F408950A2609F4A140A6958FEF0D
:109A9000811D811D08950BD07BC06CD028F071D042
:109AA00018F0952309F05DC062C01124A5C081D0D3
:109AB000A0F3959FD1F3950F50E0551F629FF001E1
:109AC000729FBB27F00DB11D639FAA27F00DB11D3A
:109AD000AA1F649F6627B00DA11D661F829F2227C3
:109AE000B00DA11D621F739FB00DA11D621F839F4A
:109AF000A00D611D221F749F3327A00D611D231F20
:109B0000849F600D211D822F762F6A2F11249F576D
:109B100050408AF0E1F088234AF0EE0FFF1FBB1F90
:109B2000661F771F881F91505040A9F79E3F51052F
:109B300070F017C061C05F3FECF3983EDCF3869590
:109B400077956795B795F795E7959F5FC1F7FE2BDA
:109B5000880F911D9695879597F9089599278827DD
:109B6000089597F99F6780E870E060E008959FEF9F
:109B700080EC089500240A941616170618060906A4
:109B8000089500240A941216130614060506089573
:109B9000092E0394000C11F4882352F0BB0F40F4FB
:109BA000BF2B11F460FF04C06F5F7F4F8F4F9F4F3B
:109BB000089557FD9058440F551F59F05F3F71F0BD
:109BC0004795880F97FB991F61F09F3F79F0879524
:109BD0000895121613061406551FF2CF4695F1DFAD
:109BE00008C0161617061806991FF1CF869571053D
:109BF000610508940895E894BB2766277727CB0171
:109C000097F90895F999FECF92BD81BDF89A9927E9
:109C100080B50895262FF999FECF1FBA92BD81BD58
:109C200020BD0FB6F894FA9AF99A0FBE01960895DE
:109C3000052E97FB16F400940FD057FD05D024D0C5
:109C400007FC02D046F408C0509540953095219508
:109C50003F4F4F4F5F4F0895909580957095619558
:109C60007F4F8F4F9F4F089531D0A59F900DB49F88
:109C7000900DA49F800D911D11240895B7FFF4CF7E
:109C8000F3DF821B930B0895A1E21A2EAA1BBB1BC4
:109C9000FD010DC0AA1FBB1FEE1FFF1FA217B307B8
:109CA000E407F50720F0A21BB30BE40BF50B661FCE
:109CB000771F881F991F1A9469F760957095809592
:109CC00090959B01AC01BD01CF010895A29FB00109
:109CD000B39FC001A39F700D811D1124911DB29FE0
:109CE000700D811D1124911D08955058BB27AA277E
:109CF0000ED04ECF3FDF30F044DF20F031F49F3FF5
:109D000011F41EF434CF0EF4E095E7FB2ACFE92FCF
:109D100050DF80F3BA17620773078407950718F0BE
:109D200071F49EF568CF0EF4E0950B2EBA2FA02D9E
:109D30000B01B90190010C01CA01A0011124FF27F8
:109D4000591B99F0593F50F4503E68F11A16F040F3
:109D5000A22F232F342F4427585FF3CF46953795F2
:109D60002795A795F0405395C9F77EF41F16BA0BB7
:109D7000620B730B840BBAF09150A1F0FF0FBB1F65
:109D8000661F771F881FC2F70EC0BA0F621F731FAE
:109D9000841F48F4879577956795B795F7959E3F0B
:109DA00008F0B3CF9395880F08F09927EE0F979599
:109DB000879508950CD0ECCEE4DE40F0DBDE30F089
:109DC00021F45F3F19F0CDCE511116CFD0CEF1DE88
:109DD00098F39923C9F35523B1F3951B550BBB2772
:109DE000AA2762177307840738F09F5F5F4F220F1F
:109DF000331F441FAA1FA9F333D00E2E3AF0E0E818
:109E000030D091505040E695001CCAF729D0FE2F63
:109E100027D0660F771F881FBB1F261737074807F5
:109E2000AB07B0E809F0BB0B802DBF01FF279358AB
:109E30005F4F2AF09E3F510568F093CEDDCE5F3F25
:109E4000ECF3983EDCF3869577956795B795F79593
:109E50009F5FC9F7880F911D9695879597F908958B
:109E6000E1E0660F771F881FBB1F62177307840727
:109E7000BA0720F0621B730B840BBA0BEE1F88F736
:109E8000E095089504D06894B111B6CE089599DE96
:109E900088F09F5790F0B92F9927B751A0F0D1F0D3
:109EA000660F771F881F991F1AF0BA95C9F712C05D
:109EB000B13081F0A0DEB1E008959DCE672F782FFC
:109EC0008827B85F39F0B93FCCF3869577956795C9
:109ED000B395D9F73EF490958095709561957F4F35
:109EE0008F4F9F4F0895B3DD08F48FEF0895AFDDD6
:109EF000880B990B0895EE0FFF1F881F8BBF0790EB
:109F0000F691E02D19946F927F928F929F92AF926B
:109F1000BF92CF92DF92EF92FF920F931F93CF9356
:109F2000DF93EC01009789F4CB01DF91CF911F9172
:109F30000F91FF90EF90DF90CF90BF90AF909F90E8
:109F40008F907F906F900C943F47FC01E60FF71FB6
:109F50009C0122503109E217F30708F4AAC0D90185
:109F60000D911C91119706171707A8F005301105E0
:109F700008F49DC0C80104978617970708F497C096
:109F800002501109061B170B019311936D937C93DB
:109F9000CF010AD88CC05B01A01AB10A4C01800E17
:109FA000911EA091E80CB091E90C40E050E0E12C4A
:109FB000F12C109709F44AC0A815B905D1F56D9098
:109FC0007C901197630182E0C80ED11CCA14DB0497
:109FD00080F1A3014A195B096A0182E0C80ED11C15
:109FE0001296BC9012971396AC91B5E0CB16D104A3
:109FF00040F0B282A38351834083D9016D937C9357
:10A000000AC00E5F1F4FC301800F911FF90191839A
:10A010008083EB2DFA2FE114F10431F0D701139670
:10A02000FC93EE93129743C0F093E90CE093E80C95
:10A030003EC08D919C9111974817590708F4AC01C7
:10A040007D0112960D90BC91A02DB3CF8091E60CAE
:10A050009091E70C88159905E1F446175707C8F465
:10A060008091020290910302009741F48DB79EB750
:10A070004091060250910702841B950BE817F907DF
:10A08000C0F4F093E70CE093E60CF9017183608370
:10A090000EC0CB010E943F477C01009751F0A80100
:10A0A000BE011CD0CE010E94D447C70104C0CE011E
:10A0B00002C080E090E0DF91CF911F910F91FF905F
:10A0C000EF90DF90CF90BF90AF909F908F907F9058
:10A0D0006F90089581E090E0F89419C0FB01DC01D5
:10A0E00002C001900D9241505040D8F70895FB01F5
:10A0F000DC018D91019080190110D9F3990B08951D
:10A10000FB01DC0101900D920020E1F7089512E0BF
:10A11000C2EAD2E000E005C0802FFE01ECDE21960D
:10A12000011DC33AD10780E00807B1F7F894FFCFCB
:10A13000FFFF0000EC0C8000200A0D000000000072
:10A14000004D178313F816000000004E17851327E3
:10A150001A00000000F3359C33A0340000000061B9
:10A160002DA92CDB2C000000009B2B3A269C2600FE
:10A17000000000950967075308000000004C358E69
:10A1800033A03300000000F2359A33D833000000CA
:10A1900000032B3826632600000000EF3594336F50
:10A1A0003400000000F032AD2C232D000000004DE3
:10A1B000359033103400000000F4359E332E350006
:10A1C0000000004E359233033500000000F1359851
:10A1D000331835000000004B358C33C634000000C6
:10A1E000005F2DA52CAF2C0000000093096307022F
:10A1F0000A00000000622DAB2C0C2D00000000F0C6
:10A20000359633933400000000602DA72C8A2C0073
:10A21000000000940965076907523033005230325C
:10A220000052303700523031005230390052383845
:10A230000052383700523838005230300052383728
:10A240000052303800523133005231320052313135
:10A250000052373300523732005237310052313713
:10A26000005231360052313500010000000100007B
:10A2700000010000005238350052383400523035A9
:10A280000052303600362E342E302E52000052301E
:10A29000340052383700000000001C258624B52405
:10A2A0006225E624C424D824000000004A358A33FD
:10A2B0005239392041524455494E4F20535441524E
:10A2C00054555020434F4D504C4554450D0A002ADB
:10A2D00000473000473030004731004730310047F9
:10A2E00032380046303900463900463131004631B7
:10A2F00032004631330046313400463135004631B4
:10A3000036004632300046323100463232004633A3
:10A310003100463332004634310046343200463490
:10A320003300463434004636310046383100463872
:10A3300032004638330046383400200A0D005239C6
:10A34000392068616E646C6572203D3D204E554C2D
:10A350004C0D0A00523939002072657365747469B6
:10A360006E67206469676974616C2070696E002093
:10A37000726573657474696E6720616E616C6F6776
:10A380002070696E0052393920484F4D45205A20BF
:10A390004F4E20535441525455500D0A00523939F2
:10A3A00020484F4D452059204F4E20535441525480
:10A3B00055500D0A0052393920484F4D452058203C
:10A3C0004F4E20535441525455500D0A00523939C2
:10A3D0002057696C6C207A65726F205800523939A9
:10A3E0002057696C6C207A65726F20590052393998
:10A3F0002057696C6C207A65726F205A0052323196
:10A400000050005600523939204572726F723A205E
:10A41000696E76616C696420706172616D657465E6
:10A42000722069640D0A0052343100686F6D650D49
:10A430000A0052393920656D657267656E6379204F
:10A4400073746F700D0A00523939206572726F7221
:10A450000D0A00523832005239392073746F70700F
:10A4600065640D0A00523939206572726F722000DE
:10A470002064656163746976617465206D6F746FC3
:10A480007220582064756520746F206D6973736540
:10A490006420737465707300206465616374697609
:10A4A000617465206D6F746F72205920647565202A
:10A4B000746F206D697373656420737465707300C5
:10A4C0002064656163746976617465206D6F746F73
:10A4D00072205A2064756520746F206D69737365EE
:10A4E00064207374657073005239392074696D6526
:10A4F0006F7574205820617869730D0A00523939DC
:10A500002074696D656F7574205920617869730DC9
:10A510000A005239392074696D656F7574205A20AC
:10A52000617869730D0A00205100523831002058BB
:10A530004100205842002059410020594200205A31
:10A540004100205A4200207374612000206375721C
:10A55000200020656E6420002068616C6620002069
:10A560006C656E2000206D696E2000206D61782082
:10A5700000207370642000523230005238332000C3
:10A580005239392043616C6962726174696F6E205F
:10A590006572726F723A20696E76616C69642061CF
:10A5A0007869732073656C65637465640D0A0020B7
:10A5B000617869732000206174207374617274691A
:10A5C0006E6720706F696E740052323300206361D1
:10A5D0006C6962726174696E67206C656E6774681D
:10A5E00000207374657020636F756E743A2000529A
:10A5F0003939206D6F76656D656E7420646F6E6598
:10A600000D0A0020617420656E6420706F696E749D
:10A61000005239392043616C6962726174696F6EEE
:10A62000206572726F723A20656E642073746F7069
:10A6300020616374697665206265666F7265207358
:10A64000746172740D0A00206D6F766520746F203E
:10A65000737461727420666F722063616C696272D8
:10A660006174696F6E006E616E00696E66006F7670
:02A67000660082
:00000001FF
